:1000000016C3000033C3000031C300002FC300003B
:100010002DC300002BC3000029C3000027C300002C
:1000200025C3000023C3000021C300001FC300003C
:100030000C9452431BC3000019C3000017C30000F7
:1000400015C3000013C300000C943E430FC300000F
:100050000DC300000BC3000009C3000007C300006C
:1000600005C3000003C3000001C30000FFC200007D
:10007000FDC20000FBC20000F9C20000F7C2000090
:10008000F5C20000F3C20000F1C20000390A4A0ABA
:100090005B0A6C0A7D0A8E0A9F0AB00A080F1A0FC3
:1000A0002C0F3E0F500F620F740F860F9A14A3147B
:1000B000AC14B514BE14C714D014D914C82025210B
:1000C00050217B218421AF21DA210522DD20E62089
:1000D000EF20F82001210A2113211C2157276F2727
:1000E0008927A327BB27D327FB2713282B28222ABE
:1000F000B62AC72B572C662D7F2E632F49305831D7
:10010000C8313832AD3219338533E433EC33F4334C
:10011000FC3304340C3414341C34ED3609372537E1
:1001200042375E377A379637B23701380A38133894
:100130001C3825382E3837384038A3382639A939A5
:10014000373AC53A443BC73B4A3CCD3C483DBA3DB3
:10015000393EC63E523F000000000000000004048B
:100160000404000400000A0A0A00000000000A0A51
:100170001F0A1F0A0A00040F140E051E0400181996
:100180000204081303000C12140814120D000C04CE
:100190000800000000000204080808040200080427
:1001A0000202020408000004150E150400000004F9
:1001B000041F04040000000000000C0408000000FC
:1001C000001F0000000000000000000C0C000001F7
:1001D0000204081000000E11131519110E00040C72
:1001E000040404040E000E11010204081F001F0283
:1001F000040201110E0002060A121F0202001F1063
:100200001E0101110E000608101E11110E001F0123
:100210000204080808000E11110E11110E000E1133
:10022000110F01020C000001020408100000000C74
:100230000C000C040800020408100804020000006E
:100240001F001F00000008040201020408000E1134
:100250000102040004000E11010D15150E000E110F
:1002600011111F1111001E11111E11111E000E116E
:10027000101010110E001C12111111121C001F1071
:10028000101E10101F001F10101E101010000E1155
:10029000101711110E001111111F111111000E0470
:1002A000040404040E000702020202120C001112E0
:1002B0001418141211001010101010101F00111B30
:1002C00015151111110011111915131111000E112D
:1002D000111111110E001E11111E101010000E111F
:1002E000111115120D001E11111E141211000F1004
:1002F000100E01011E001F04040404040400111167
:10030000111111110E0011111111110A0400111116
:10031000111115150E0011110A040A111100111105
:10032000110A040404001F01020408101F000E0833
:10033000080808080E00110A1F041F0404000E021A
:10034000020202020E00040A110000000000000078
:10035000000000001F000804000000000000000072
:100360000E010F110F0010101E1111111E000000C0
:100370000E1010110E0001010D1311110F000000DD
:100380000E111F100E000609081C08080800000FB7
:1003900011110F010E001010161911111100040097
:1003A0000C0404040E000200060202120C001010DD
:1003B0001214181412001808080808081C0000007D
:1003C0001A15151111000000161911111100000065
:1003D0000E1111110E0000001E111E101000000061
:1003E0000F110F010100000016191010100000007D
:1003F0000E100E011E0008081C0808090600000067
:10040000111111130D0000001111110A0400000058
:10041000111111150A000000110A040A1100000050
:1004200011110F010E0000001F0204081F003844C4
:1004300044447C4444007C40407844447800784400
:100440004478444478007C404040404040000C14D4
:10045000242424243C447C40407840407C00545474
:100460005438545454003844041804443800444464
:100470004C546444440054444C5464444400444840
:100480005060504844001C24242424246400446CFC
:100490005454444444004444447C44444400384458
:1004A0004444444438007C44444444444400784434
:1004B00044784040400038444040404438007C107C
:1004C0001010101010004444443C044438003854C8
:1004D0005454381010004444281028444400444424
:1004E000444444447E02444444443C040400545480
:1004F000545454547C005454545454547E02602038
:100500002038242438004444446454546400404057
:100510004078444478003844041C0444380048546B
:100520005474545448003C44443C14244400000097
:1005300038043C443C0000007840784478000000D7
:10054000784C784C78000000784040404000000033
:10055000182828287C44000038447C403C000000D7
:1005600054543854540000007804380478000000D3
:10057000444C546444000010444C54644400000053
:1005800044487048440000001C24444444000000D7
:10059000446C545444000000484878484800000027
:1005A0003844444438000000784848484800000077
:1005B0007048704040000000384040403800000063
:1005C0007C1010101000000048483808700000002F
:1005D000385454381000000044281028440000000B
:1005E000484848487C040000484838080800000093
:1005F000545454547C000000545454547E0200005F
:1006000060203C223C0000004242724A720000001E
:1006100040407844780000007008780870000000BE
:100620004C5272524C0000003C443C4444001124A3
:100630001FBECFEFD0E1DEBFCDBF15E0A0E0B1E03F
:10064000ECECF3E900E00BBF02C007900D92A03D77
:10065000B107D9F726E0A0EDB5E001C01D92AE3795
:10066000B207E1F70E94B0430C94E449C9CCE2E63A
:10067000F0E090819E7F9083908194609083908140
:10068000977F9083A8988BBB8DE08A95F1F7000047
:10069000A89A8081886080830895E2E6F0E09081E6
:1006A000916090839081946090839081977F9083F4
:1006B000A8988BBB8DE08A95F1F70000A89A8081FD
:1006C000886080830895CF93C82F892FE6DF8C2F11
:1006D000E4DFCF910895E2E6F0E0208121602083FD
:1006E0002081246020832081277F2083A8988BBBD2
:1006F00092BB8DE08A95F1F70000A89A808188600E
:1007000080830895CF93C82F86E3B1DFC13049F0CD
:1007100028F0C23049F0C33051F00CC088E4BDDF8E
:100720000BC088E2BADF15C088E8B7DF05C088EEE5
:10073000B4DF0FC0CD7F69F48FEE90E09093D305C6
:100740008093D2058FE391E09093D1058093D005FB
:100750000CC08FE391E09093D3058093D2058FEE88
:1007600090E09093D1058093D005CF910895CF93D9
:10077000C82F8FEF8ABB81BB8093610081E084BB6F
:10078000E2E6F0E080818260808381E070DF2FEF1D
:1007900089E698E1215080409040E1F700C00000D8
:1007A00080EC65DF85E279DF81EC61DF81E175DF77
:1007B00085EC5DDF8BE271DF8BE26FDF87EC57DF6B
:1007C00086E86BDF8C2F9EDF8AE351DF85E065DFF3
:1007D00081EB4DDF80E061DF88E15FDF86EB47DFA3
:1007E0008AE05BDF82E859DF87E257DF81E13FDFA4
:1007F0002FEF8DEE92E0215080409040E1F700C055
:10080000000089E234DFCF9108950F931F93CF93B7
:10081000DF938C01EB018AE22ADFC80154DFCE01AD
:1008200052DFDF91CF911F910F9108950F931F9386
:10083000CF93DF938C01EB018BE219DFC80143DF1B
:10084000CE0141DFDF91CF911F910F910895CF939A
:10085000DF93EB01BC01D9DFBE01CE01E7DF8CE203
:1008600006DFDF91CF910895CF93DF93EA01EFDFA9
:10087000CE0131DFDF91CF9108958F929F92AF9299
:10088000BF92CF92DF92EF92FF920F931F93CF937D
:10089000DF93A8956817790738F486279727682784
:1008A000792786279727A8952417350738F44227F4
:1008B00053272427352742275327A895A091D205EF
:1008C000B091D305FC01A817B90708F4FD01EB01AD
:1008D000A617B70708F4ED018091D0059091D105D6
:1008E0007A018417950708F47C0169018217930740
:1008F00008F46C01A8959E012F5F3F4F2E1B3F0B04
:10090000D6011196AE19BF090E94AC464B015C019D
:10091000BE01CF017ADFA895B601C70187DF8CE25F
:10092000A6DEA89581149104A104B10481F0C12C24
:10093000D12C7601C801CFDEA8958FEFC81AD80A4E
:10094000E80AF80A8C149D04AE04BF0499F7DF91FD
:10095000CF911F910F91FF90EF90DF90CF90BF90BC
:10096000AF909F908F9008950F931F93411551055D
:1009700079F02115310561F0FA01AB01615071097F
:10098000260F371FBC01615071096E0F7F1F75DF85
:100990001F910F9108952F923F924F925F926F9205
:1009A0007F928F929F92AF92BF92CF92DF92EF92FF
:1009B000FF920F931F93CF93DF93CDB7DEB761976D
:1009C0000FB6F894DEBF0FBECDBF8B879C875887CC
:1009D0004F833A8729870D872E2C312C802F90E06A
:1009E0009C01220F331F220F331F220F331FA90137
:1009F000425D51405C834B83F901EA5CF140FF8723
:100A0000EE87662E772E21015FC07720ECF0ED8116
:100A1000FE81849190E0088802C0959587950A949C
:100A2000E2F780FF09C00F8118859101A10169815A
:100A30007A81C70199DF08C009851A859101A10152
:100A400069817A81C60190DFFFEBF715E8F4EB814D
:100A5000FC81849190E0088802C0959587950A945E
:100A6000E2F780FF09C00F8118859101A10169811A
:100A70007A81C40179DF08C009851A859101A10135
:100A800069817A81C50170DF840C951CA40CB51CAA
:100A90002889398921503109398B288BE40CF51CC0
:100AA000C40CD51C2F3F3F4F09F0AFCF69807A802F
:100AB000620C731C8B819C8101969C838B83EE85D9
:100AC000FF858E179F07B1F0CB84DC84EC2CFD2CC6
:100AD000AC2CBD2C8C2C9D2C27E030E04B815C8114
:100AE000485D5D4F5E834D837A826982398B288BA6
:100AF0007D848BCF61960FB6F894DEBF0FBECDBF5D
:100B0000DF91CF911F910F91FF90EF90DF90CF90E9
:100B1000BF90AF909F908F907F906F905F904F901D
:100B20003F902F9008954F925F926F927F928F9295
:100B30009F92AF92BF92CF92DF92EF92FF920F936C
:100B40001F93CF93DF93EC015B012A013901102F32
:100B5000F7010081002331F1812E912C880C991C22
:100B6000880C991C880C991C6701FFEFCF1ADF0ACB
:100B70002091D2053091D305CE0108962817390768
:100B800020F4A80CB91CC1E0D0E0E12E9301A20131
:100B9000B501CE0100DFC80DD91DF60101916F012D
:100BA0000111E6CFDF91CF911F910F91FF90EF9050
:100BB000DF90CF90BF90AF909F908F907F906F907D
:100BC0005F904F9008956F927F928F929F92AF9215
:100BD000BF92CF92DF92EF92FF920F93CF93DF936A
:100BE00000D000D0CDB7DEB76C015B014A013901FE
:100BF000C70119821A821B821C824AE0BE016F5F04
:100C00007F4F0E94BB46CE0101967C019301A40157
:100C1000B501C60188DF0F900F900F900F90DF9104
:100C2000CF910F91FF90EF90DF90CF90BF90AF905A
:100C30009F908F907F906F9008950F931F932091B6
:100C4000D0053091D1056091D2057091D3058C010A
:100C500040E050E080E090E010DE1F910F91089599
:100C6000EF92FF920F931F93CF93DF93EB018A01D3
:100C70007901BC01640F751FC8DDBE01CE01D6DD50
:100C80008CE2F5DC0115110541F0C0E0D0E0C701B0
:100C900022DD2196C017D107D1F7DF91CF911F91A7
:100CA0000F91FF90EF900895EF92FF920F931F9393
:100CB000CF93DF93EB018A017901BC01A6DDBE0170
:100CC000600F711FCE01B2DD8CE2D1DC0115110580
:100CD00041F0C0E0D0E0C701FEDC2196C017D1078B
:100CE000D1F7DF91CF911F910F91FF90EF90089571
:100CF0002F923F924F925F926F927F928F929F922C
:100D0000AF92BF92CF92DF92EF92FF920F931F9319
:100D1000CF93DF9300D000D000D0CDB7DEB79E8355
:100D20008D837B013A0129011A830983C901861B3E
:100D3000970B9A014D815E81241B350B890122F4AA
:100D400000271127021B130B2D813E812615370525
:100D500020F0AA24AA94BA2C03C0AA24A394B12CEC
:100D60006C01992324F4CC24DD24C81AD90ADC822E
:100D7000CB82D194C194D108E414F50420F08824E6
:100D80008A94982C03C088248394912C18014B8159
:100D90005C81241A350A49815A81B7018D819E816F
:100DA00063DDC101880F991F8C159D056CF02D81A5
:100DB0003E812615370599F04B815C81241A350A4E
:100DC0002A0D3B1D3E832D830817190724F3E414D5
:100DD000F50429F0200E311EE80CF91CDCCF269614
:100DE0000FB6F894DEBF0FBECDBFDF91CF911F913C
:100DF0000F91FF90EF90DF90CF90BF90AF909F90BA
:100E00008F907F906F905F904F903F902F900895BC
:100E1000AF92BF92CF92DF92EF92FF920F931F9308
:100E2000CF93DF937C016B01EA015901980118DF30
:100E3000B501615071096C0D7D1D9801AE01C701AE
:100E40000FDF9801A501B601C7012EDFCE01019782
:100E50009801A501B6018E0D9F1D26DFDF91CF9170
:100E60001F910F91FF90EF90DF90CF90BF90AF90C8
:100E700008952F923F924F925F926F927F928F923E
:100E80009F92AF92BF92CF92DF92EF92FF920F9319
:100E90001F93CF93DF934C015B01190150E00027B2
:100EA0001127041B150BC1E0D0E0C41BD50BCC0FE0
:100EB000DD1FE12CF12CA1016701CA0CDB1CB6017E
:100EC0002401401A510AC201CFDCA101B601680118
:100ED000C80CD91CC601C8DCA10135016E187F08F9
:100EE000B301C601C1DCA101B301C201BDDCEC1636
:100EF000FD06BCF02FEFE21AF20AC701880F991F16
:100F000001968C0F9D1F22273327201B310BE216E1
:100F1000F30641F40C171D0744F020E0C22FD22F36
:100F200001C0CE010C171D074CF40F5F1F4FE801E5
:100F3000CC0FDD1F2196C80FD91F01C0EC01101680
:100F400011060CF0B8CFDF91CF911F910F91FF9058
:100F5000EF90DF90CF90BF90AF909F908F907F9059
:100F60006F905F904F903F902F9008954F925F92B7
:100F70006F927F928F929F92AF92BF92CF92DF92A9
:100F8000EF92FF920F931F93CF93DF93EC015B01DE
:100F90004A01390128018601ABDE9701A201B301A4
:100FA000C401A6DE9501AE01B701C201A1DEDF9149
:100FB000CF911F910F91FF90EF90DF90CF90BF9056
:100FC000AF909F908F907F906F905F904F9008951B
:100FD000CF93C82F8A3011F48DE0FADF5D9BFECFEE
:100FE000CCB980E090E0CF910895CF92DF92EF925C
:100FF000FF920F931F93A8950FEF1FEF21E430E0AE
:101000004FE550E065E070E085E090E001DFA895F5
:1010100021E430E04FE550E06BE470E085E090E0E3
:10102000F7DE2BE430E04FE550E061E970E085E069
:1010300090E0EEDE0F2EFDE1EF2EF5E0FF2EF02D1D
:1010400001E02FE130E04FEF5FEF60E570E082E11B
:1010500090E069DD0F2EF8E1EF2EF5E0FF2EF02D88
:101060002FE130E04FEF5FEF6AE570E083E290E060
:101070005ADD0FEF1FEF21E430E04FE550E065E06F
:1010800070E08CED90E0C4DE21E430E04FE550E00C
:101090006BE470E08CED90E0BBDE2BE430E04FE5DC
:1010A00050E061E970E08CED90E0B2DE0F2EFDE1E2
:1010B000EF2EF5E0FF2EF02D01E02FE130E04FEFB5
:1010C0005FEF60E570E08BEE90E02DDD0F2EF2E13A
:1010D000EF2EF5E0FF2EF02D2FE130E04FEF5FEF28
:1010E0006AE570E08CEF90E01EDDA89580910A061D
:1010F00090910B06019709F053C00FE110E024E432
:1011000030E048E550E064E970E088E090E02CDCF5
:101110002CE430E04EE650E06CE870E089E690E0C8
:1011200023DC24E430E048E550E064E970E080EE40
:1011300090E01ADC20EE37E048E264EB70E080EAF1
:1011400090E097DE20EE37E047E264EB70E080EA63
:1011500090E08FDE20EE37E04BE264EB70E080EA57
:1011600090E087DE20EE37E045E264EB70E080EA55
:1011700090E07FDE0F2EF0EECF2EF7E0DF2EF02D89
:101180000F2EF4EBEF2EF12CF02D07EB10E028ECF6
:1011900030E044E950E060EA70E084E990E0E6DEA7
:1011A000A89580910A0690910B06892B09F051C0F1
:1011B0000FE110E024E430E048E550E064E970E03D
:1011C00088E090E0D1DB2CE430E04EE650E06CE8C3
:1011D00070E089E690E0C8DB24E430E048E550E0C8
:1011E00064E970E080EE90E0BFDB20E038EF48E299
:1011F00064EB70E080EA90E03CDE20E038EF47E20C
:1012000064EB70E080EA90E034DE20E038EF4BE2FF
:1012100064EB70E080EA90E02CDE20E038EF45E2FD
:1012200064EB70E080EA90E024DE00E018EF23E257
:1012300030E045E050E065EA70E086E990E094DB5C
:1012400023E230E045E050E065EA70E085EA90E0B6
:101250008BDBA89580910C0690910D06892B89F463
:10126000A8950F2EF8E0EF2EF5E0FF2EF02D01E00F
:101270002FE130E04FEF5FEF63E270E08AE090E053
:1012800052DC80910C0690910D06019701F5A8950E
:101290000F2EF1ECEF2EF5E0FF2EF02D01E02FE107
:1012A00030E04FEF5FEF64E170E084E190E03BDC21
:1012B0000F2EFBEBEF2EF5E0FF2EF02D2FE130E0AF
:1012C0004FEF5FEF68E270E08EE190E02CDCA895D4
:1012D00080910C0690910D06029701F5A8950F2EAE
:1012E000F4EBEF2EF5E0FF2EF02D01E02FE130E0E2
:1012F0004FEF5FEF64E170E084E190E014DC0F2ECB
:10130000FBEBEF2EF5E0FF2EF02D2FE130E04FEF5D
:101310005FEF68E270E08EE190E005DCA8958091D7
:101320000C0690910D06039789F4A8950F2EFDEAFF
:10133000EF2EF5E0FF2EF02D01E02FE130E04FEF32
:101340005FEF63E270E089E190E0EDDBA8958091CA
:101350000C0690910D06049789F4A8950F2EFEECCB
:10136000EF2EF4E0FF2EF02D01E02FE130E04FEF03
:101370005FEF63E270E08FE090E0D5DBA8958091AD
:101380000C0690910D06059701F5A8950F2EF8EC27
:10139000EF2EF4E0FF2EF02D01E02FE130E04FEFD3
:1013A0005FEF64E170E089E190E0BDDB0F2EFEEBC2
:1013B000EF2EF4E0FF2EF02D2FE130E04FEF5FEF46
:1013C00063E270E08FE090E0AEDBA89580910C06C0
:1013D00090910D06069701F5A8950F2EF8ECEF2ECB
:1013E000F4E0FF2EF02D01E02FE130E04FEF5FEF52
:1013F00064E170E089E190E096DB0F2EFCEAEF2ECD
:10140000F4E0FF2EF02D2FE130E04FEF5FEF63E2CD
:1014100070E08FE190E087DBA89580910C069091B9
:101420000D06079789F4A8950F2EF3E9EF2EF4E047
:10143000FF2EF02D01E02FE130E04FEF5FEF63E290
:1014400070E08FE090E06FDB80910C0690910D06CC
:10145000892B09F095C0A895E09169068E2F90E040
:101460008830910508F08CC0FC01EA5BFF4F0C94BA
:10147000A3460F2EFEE8EF2EF4E0FF2EF02D02E043
:101480002FE130E04FEF5FEF6EE170E08BEE90E028
:101490004ADB76C00F2EF9E8EF2EF4E0FF2EF02D98
:1014A00002E02FE130E04FEF5FEF6EE170E08BEE96
:1014B00090E039DB65C00F2EFFE7EF2EF4E0FF2E42
:1014C000F02D01E02FE130E04FEF5FEF6EE170E0D3
:1014D00086EE90E028DB54C00F2EF5E7EF2EF4E007
:1014E000FF2EF02D01E02FE130E04FEF5FEF6EE1D6
:1014F00070E086EE90E017DB43C00F2EFBE6EF2E88
:10150000F4E0FF2EF02D01E02FE130E04FEF5FEF30
:101510006EE170E086EE90E006DB32C00F2EF1E661
:10152000EF2EF4E0FF2EF02D01E02FE130E04FEF41
:101530005FEF6EE170E086EE90E0F5DA21C00F2EED
:10154000F7E5EF2EF4E0FF2EF02D01E02FE130E083
:101550004FEF5FEF6EE170E086EE90E0E4DA10C0EE
:101560000F2EFDE4EF2EF4E0FF2EF02D01E02FE131
:1015700030E04FEF5FEF6EE170E086EE90E0D3DA9F
:1015800080910C0690910D06019709F03BC0A8953B
:10159000809115068130A9F018F0823019F132C01F
:1015A0000F2EFFE7EF2EF4E0FF2EF02D01E02FE1EC
:1015B00030E04FEF5FEF6EE170E086EE90E0B3DA7F
:1015C00021C00F2EF5E7EF2EF4E0FF2EF02D01E005
:1015D0002FE130E04FEF5FEF6EE170E086EE90E0DC
:1015E000A2DA10C00F2EFBE6EF2EF4E0FF2EF02D56
:1015F00001E02FE130E04FEF5FEF6EE170E086EE4B
:1016000090E091DA80910C0690910D06029709F016
:101610003BC0A89580911C068130A9F018F082305B
:1016200019F132C00F2EFFE7EF2EF4E0FF2EF02D60
:1016300001E02FE130E04FEF5FEF6EE170E086EE0A
:1016400090E071DA21C00F2EF5E7EF2EF4E0FF2EC7
:10165000F02D01E02FE130E04FEF5FEF6EE170E041
:1016600086EE90E060DA10C00F2EFBE6EF2EF4E07D
:10167000FF2EF02D01E02FE130E04FEF5FEF6EE144
:1016800070E086EE90E04FDA80910C0690910D06A6
:10169000039789F4A8950F2EF9EDEF2EF4E0FF2EB5
:1016A000F02D01E02FE130E04FEF5FEF6EE170E0F1
:1016B0008EEE90E038DA80910C0690910D0604973A
:1016C00009F03BC0A895809174068130A9F018F00C
:1016D000823019F132C00F2EFFE7EF2EF4E0FF2E1B
:1016E000F02D01E02FE130E04FEF5FEF6EE170E0B1
:1016F00086EE90E018DA21C00F2EF5E7EF2EF4E029
:10170000FF2EF02D01E02FE130E04FEF5FEF6EE1B3
:1017100070E086EE90E007DA10C00F2EFBE6EF2EA9
:10172000F4E0FF2EF02D01E02FE130E04FEF5FEF0E
:101730006EE170E086EE90E0F6D980910C06909113
:101740000D06059709F03BC0A89580916806813089
:10175000A9F018F0823019F132C00F2EFFE7EF2EFA
:10176000F4E0FF2EF02D01E02FE130E04FEF5FEFCE
:101770006EE170E086EE90E0D6D921C00F2EF5E73D
:10178000EF2EF4E0FF2EF02D01E02FE130E04FEFDF
:101790005FEF6EE170E086EE90E0C5D910C00F2ECD
:1017A000FBE6EF2EF4E0FF2EF02D01E02FE130E01C
:1017B0004FEF5FEF6EE170E086EE90E0B4D980917C
:1017C0000C0690910D06069709F03BC0A8958091F4
:1017D00065068130A9F018F0823019F132C00F2E61
:1017E000FFE7EF2EF4E0FF2EF02D01E02FE130E0D7
:1017F0004FEF5FEF6EE170E086EE90E094D921C08C
:101800000F2EF5E7EF2EF4E0FF2EF02D01E02FE193
:1018100030E04FEF5FEF6EE170E086EE90E083D94D
:1018200010C00F2EFBE6EF2EF4E0FF2EF02D01E0AE
:101830002FE130E04FEF5FEF6EE170E086EE90E079
:1018400072D980910C0690910D06079709F4A8951E
:101850001F910F91FF90EF90DF90CF900895CF925E
:10186000DF92EF92FF920F931F93A89500EE17E07F
:1018700021E430E048EC50E06AEA70E085E090E076
:1018800073D80FEF1FEF21E430E048EC50E063E243
:1018900070E085E090E0BCDA0F2EF1E6EF2EF2E08A
:1018A000FF2EF02D01E02FE130E040EE57E06CE339
:1018B00070E088E290E037D90FEF1FEF20E530E0CD
:1018C00040E550E065E070E08BEE90E0A1DA0F2E8D
:1018D000F0EECF2EF7E0DF2EF02D0F2EF4E1EF2EFD
:1018E000F12CF02D03E111E026E430E041E351E07A
:1018F00066E470E085EF90E039DB0F2EF7E1EF2E24
:10190000F12CF02D24E430E04FE251E064E470E08B
:1019100087EF90E02BDB0FEF1FEF20E530E040E595
:1019200050E064E670E08BEE90E072DA0F2EF5EA9C
:10193000EF2EF12CF02D03E111E023E730E041E33D
:1019400051E063E770E085EF90E010DB0F2EF3EAE3
:10195000EF2EF12CF02D25E730E04FE251E065E766
:1019600070E087EF90E002DB0F2EF0E3EF2EF5E062
:10197000FF2EF02D02E020EE37E040E050E068EC72
:1019800070E08DE290E0CFD81F910F91FF90EF9023
:10199000DF90CF900895CF92DF92EF92FF920F9356
:1019A0001F93A89500EE17E021E430E048EC50E0EA
:1019B0006AEA70E085E090E00E94B4040FEF1FEF48
:1019C00021E430E048EC50E063E270E085E090E034
:1019D0001FDA0F2EFDE9EF2EF4E0FF2EF02D01E0CF
:1019E0002FE130E040EE57E06CE370E088E290E0F9
:1019F0009AD80FEF1FEF20E530E040E550E065E0BA
:101A000070E08BEE90E004DA0F2EF0EECF2EF7E0D0
:101A1000DF2EF02D0F2EF4E1EF2EF12CF02D03E14F
:101A200011E026E430E041E351E066E470E085EF48
:101A300090E09CDA0F2EF7E1EF2EF12CF02D24E44C
:101A400030E04FE251E064E470E087EF90E08EDA3E
:101A50000FEF1FEF20E530E040E550E064E670E076
:101A60008BEE90E0D5D90F2EF5EAEF2EF12CF02D6C
:101A700003E111E023E730E041E351E063E770E088
:101A800085EF90E073DA0F2EF3EAEF2EF12CF02DB4
:101A900025E730E04FE251E065E770E087EF90E046
:101AA00065DA0F2EF9ECEF2EF5E0FF2EF02D02E0B7
:101AB00020EE37E040E050E068EC70E08DE290E02E
:101AC00032D81F910F91FF90EF90DF90CF90089543
:101AD000CF92DF92EF92FF920F931F93A89500EEA3
:101AE00017E021E430E048EC50E06AEA70E085E07D
:101AF00090E00E94B4040FEF1FEF21E430E048ECC7
:101B000050E063E270E085E090E082D90F2EFCE3C4
:101B1000EF2EF4E0FF2EF02D01E02FE130E040EE5B
:101B200057E06CE370E088E290E00E9493050FEFCD
:101B30001FEF20E530E040E550E065E070E08BEE1F
:101B400090E066D90F2EF0EECF2EF7E0DF2EF02DCD
:101B50000F2EF4E1EF2EF12CF02D03E111E026E43D
:101B600030E041E351E066E470E085EF90E0FED9BB
:101B70000F2EF7E1EF2EF12CF02D24E430E04FE2B0
:101B800051E064E470E087EF90E0F0D90FEF1FEFD1
:101B900020E530E040E550E064E670E08BEE90E058
:101BA00037D90F2EF5EAEF2EF12CF02D03E111E0DD
:101BB00023E730E041E351E063E770E085EF90E038
:101BC000D5D90F2EF3EAEF2EF12CF02D25E730E0DA
:101BD0004FE251E065E770E087EF90E0C7D90F2E44
:101BE000F1E4EF2EF5E0FF2EF02D02E020EE37E0DD
:101BF00040E050E068EC70E08DE290E00E949305D8
:101C00001F910F91FF90EF90DF90CF900895CF93A9
:101C1000DF9300D000D0CDB7DEB7809163001C8287
:101C20001B821A821982BE016F5F7F4FCE0103961D
:101C30000E9418458B819C81853C994068F0898180
:101C40009A81843A964040F489819A818D329140FC
:101C500018F082E0809334068B819C81803D974010
:101C600090F48B819C818139914068F089819A81BF
:101C7000843A964040F489819A818D32914018F0DF
:101C800083E0809334068B819C818032934068F49A
:101C900089819A8184379E4040F489819A81813D6F
:101CA000974018F081E0809334068B819C81843CBE
:101CB000994060F48B819C81893E934038F0898102
:101CC0009A81813D974010F010923406809134063D
:101CD0000F900F900F900F90DF91CF910895CF92BA
:101CE000DF92EF92FF920F931F93A89500EE17E0FB
:101CF00021E430E048EC50E06AEA70E085E090E0F2
:101D00000E94B4040FEF1FEF21E430E048EC50E0F4
:101D100063E270E085E090E07BD820E530E040E5CC
:101D200050E065E070E08BEE90E072D80F2EF0EEA0
:101D3000CF2EF7E0DF2EF02D0F2EF4E1EF2EF12C59
:101D4000F02D03E111E026E430E041E351E066E4E8
:101D500070E085EF90E00AD90F2EF7E1EF2EF12C1D
:101D6000F02D24E430E04FE251E064E470E087EFCE
:101D700090E0FCD80FEF1FEF20E530E040E550E0A9
:101D800064E670E08BEE90E043D80F2EF5EAEF2E7C
:101D9000F12CF02D03E111E023E730E041E351E0C5
:101DA00063E770E085EF90E0E1D80F2EF3EAEF2EC5
:101DB000F12CF02D25E730E04FE251E065E770E0CF
:101DC00087EF90E0D3D80F2EF9ECEF2EF5E0FF2E41
:101DD000F02D02E020EE37E040E050E068EC70E0EB
:101DE0008CE390E00E94930580910C0690910D0683
:101DF000892B09F09CC0E09169068E2F90E0883015
:101E0000910508F094C0FC01E25BFF4F0C94A346DF
:101E10000F2EFEE8EF2EF4E0FF2EF02D02E02FE172
:101E200030E04FEF5FEF65E070E086E490E00E9405
:101E300093057DC00F2EF9E8EF2EF4E0FF2EF02D74
:101E400002E02FE130E04FEF5FEF65E070E086E405
:101E500090E00E9493056BC00F2EFFE7EF2EF4E099
:101E6000FF2EF02D02E02FE130E04FEF5FEF65E055
:101E700070E08EE190E00E94930559C00F2EF5E7C7
:101E8000EF2EF4E0FF2EF02D02E02FE130E04FEFD7
:101E90005FEF65E070E08EE190E00E94930547C03F
:101EA0000F2EFBE6EF2EF4E0FF2EF02D02E02FE1E7
:101EB00030E04FEF5FEF65E070E08EE190E00E9470
:101EC000930535C00F2EF1E6EF2EF4E0FF2EF02D36
:101ED00002E02FE130E04FEF5FEF65E070E08EE170
:101EE00090E00E94930523C00F2EF7E5EF2EF4E05B
:101EF000FF2EF02D02E02FE130E04FEF5FEF65E0C5
:101F000070E08EE190E00E94930511C00F2EFDE479
:101F1000EF2EF4E0FF2EF02D02E02FE130E04FEF46
:101F20005FEF65E070E08EE190E00E9493058091A4
:101F30000C0690910D060197E9F580911506813008
:101F4000B1F018F0823029F135C00F2EFFE7EF2EE7
:101F5000F4E0FF2EF02D02E02FE130E04FEF5FEFD5
:101F600065E070E08EE190E00E94930523C00F2EA3
:101F7000F5E7EF2EF4E0FF2EF02D02E02FE130E048
:101F80004FEF5FEF65E070E08EE190E00E94930517
:101F900011C00F2EFBE6EF2EF4E0FF2EF02D02E035
:101FA0002FE130E04FEF5FEF65E070E08EE190E011
:101FB0000E94930580910C0690910D060297E9F519
:101FC00080911C068130B1F018F0823029F135C0C3
:101FD0000F2EFFE7EF2EF4E0FF2EF02D02E02FE1B1
:101FE00030E04FEF5FEF65E070E08EE190E00E943F
:101FF000930523C00F2EF5E7EF2EF4E0FF2EF02D12
:1020000002E02FE130E04FEF5FEF65E070E08EE13E
:1020100090E00E94930511C00F2EFBE6EF2EF4E036
:10202000FF2EF02D02E02FE130E04FEF5FEF65E093
:1020300070E08EE190E00E94930580910C069091F3
:102040000D060497E9F5809174068130B1F018F01F
:10205000823029F135C00F2EFFE7EF2EF4E0FF2E7E
:10206000F02D02E02FE130E04FEF5FEF65E070E030
:102070008EE190E00E94930523C00F2EF5E7EF2E2E
:10208000F4E0FF2EF02D02E02FE130E04FEF5FEFA4
:1020900065E070E08EE190E00E94930511C00F2E84
:1020A000FBE6EF2EF4E0FF2EF02D02E02FE130E012
:1020B0004FEF5FEF65E070E08EE190E00E949305E6
:1020C00080910C0690910D060597E9F580916806C0
:1020D0008130B1F018F0823029F135C00F2EFFE7C2
:1020E000EF2EF4E0FF2EF02D02E02FE130E04FEF75
:1020F0005FEF65E070E08EE190E00E94930523C001
:102100000F2EF5E7EF2EF4E0FF2EF02D02E02FE189
:1021100030E04FEF5FEF65E070E08EE190E00E940D
:10212000930511C00F2EFBE6EF2EF4E0FF2EF02DED
:1021300002E02FE130E04FEF5FEF65E070E08EE10D
:1021400090E00E94930580910C0690910D060697F1
:10215000E9F5809165068130B1F018F0823029F1FF
:1021600035C00F2EFFE7EF2EF4E0FF2EF02D02E03A
:102170002FE130E04FEF5FEF65E070E08EE190E03F
:102180000E94930523C00F2EF5E7EF2EF4E0FF2EFB
:10219000F02D02E02FE130E04FEF5FEF65E070E0FF
:1021A0008EE190E00E94930511C00F2EFBE6EF2E0A
:1021B000F4E0FF2EF02D02E02FE130E04FEF5FEF73
:1021C00065E070E08EE190E00E9493051F910F9111
:1021D000FF90EF90DF90CF900895EF92FF920F93D2
:1021E0001F9380910306909104068A30910508F0B0
:1021F0007BC08091DC0581110CC00FE110E02CE365
:1022000030E044E650E06BE470E08EE690E00E943F
:10221000B40481E08093DC0510920E0680910306E1
:10222000909104068436910580F50A9790F104C0D8
:1022300080910E0681110CC00FE110E02CE330E01C
:1022400044E650E06BE470E08EE690E00E94B40457
:1022500081E080930E061092DC0580910306909138
:10226000040684369105A8F004C080910E068130E2
:1022700061F40FE110E02CE330E044E650E06BE461
:1022800070E08EE690E00E94B40410920E06109268
:10229000DC0580910A0690910B06019779F4E09095
:1022A0000306F090040603E02FE130E04FEF5FEF0C
:1022B00064E670E082E890E00E94E30580910A06FF
:1022C00090910B06892BA9F4E0900306F090040688
:1022D00003E02FE130E040E058EF64E670E082E890
:1022E00090E00E94E30505C08436910508F4A0CF74
:1022F000BCCF1F910F91FF90EF900895EF92FF9246
:102300000F931F9380913806909139060A97E8F44D
:1023100080910206811119C00FE110E027E330E03F
:1023200048E550E06BE970E088E090E00E94B4047A
:1023300081E08093020610926606809138069091A3
:1023400039068436910548F036C080913806909160
:1023500039068436910508F042C0809103069091B9
:1023600004060A9760F180916606811128C00FE18A
:1023700010E027E330E048E550E06BE970E088E0EA
:1023800090E00E94B40481E08093660610920206F9
:1023900080913806909139068436910580F00FE1DE
:1023A00010E027E330E048E550E06BE970E088E0BA
:1023B00090E00E94B4041092660610920206E0902B
:1023C0003806F090390603E02FE130E04FEF5FEF81
:1023D00064EB70E08FE090E00E94E30505C080911F
:1023E0006606813041F7DBCF1F910F91FF90EF9090
:1023F0000895EF92FF920F931F938091250690917D
:1024000026068A30910508F0B9C08091090681112D
:102410000CC00FE110E024E230E04AE550E064E651
:1024200070E088E090E00E94B40481E080930906A7
:102430001092200680912506909126060A978A35EB
:10244000910508F0A4C004C08091200681110CC041
:102450000FE110E024E230E04AE550E064E670E08D
:1024600088E090E00E94B40481E0809320061092FE
:102470000906809125069091260684369105E1F49F
:102480000BC0809125069091260684369105A1F413
:1024900080912006813061F40FE110E024E230E009
:1024A0004AE550E064E670E088E090E00E94B40401
:1024B0001092090610922006E0902506F09026065C
:1024C00003E02FE130E04FEF5FEF6EE670E084E174
:1024D00090E00E94E30580917506909176068A301F
:1024E000910508F050C080916F0681112FC00FE157
:1024F00010E024E230E04AE550E064E670E08FED61
:1025000090E00E94B40481E080936F0610923A0636
:1025100080917506909176060A978A359105B0F4F8
:1025200004C080913A06811111C00FE110E024E24D
:1025300030E04AE550E064E670E08FED90E00E9404
:10254000B40481E080933A0610926F06E09075061D
:10255000F090760684E6E816F10421F410926F06F6
:1025600010923A0603E02FE130E04FEF5FEF6EE6A6
:1025700070E089EE90E00E94E30512C08436910578
:1025800008F462CF7ECF8436910558F2DFCF809178
:102590002506909126068436910509F08DCF88CFC7
:1025A0001F910F91FF90EF900895CF93DF9300D08C
:1025B00000D0CDB7DEB7809163001C821B821A82E7
:1025C0001982BE016F5F7F4FCE0103960E941845AE
:1025D0008B819C8188379540A0F4A89589819A8148
:1025E000843C994070F4A89589819A818D3D9540ED
:1025F00040F0A89581E090E090930B0680930A0646
:10260000A8950F900F900F900F90DF91CF910895A4
:10261000CF93DF9300D000D0CDB7DEB7A8958091DF
:1026200063001C821B821A821982BE016F5F7F4F7A
:10263000CE0103960E9418458B819C818837954076
:1026400070F489819A81843C994048F489819A8107
:102650008D3D954020F010920B0610920A060F90C7
:102660000F900F900F90DF91CF9108957F928F92EE
:102670009F92AF92BF92CF92DF92EF92FF920F9311
:102680001F93CF93DF93EC016B015A014901702E28
:10269000A8958091DF059091E0058A30910508F0BA
:1026A00069C080916A06811139C00FE110E02EE106
:1026B00030E044E650E065507109CE0144970E9435
:1026C000B40481E080936A0610922D068091DF05A4
:1026D0009091E0058A30910508F151C080912D0656
:1026E00081113BC00FE110E02EE130E044E650E004
:1026F000B60165507109CE0144970E94B40481E08F
:1027000080932D0610926A06109205068091DF05CF
:102710009091E0058436910560F41FC08091DF053B
:102720009091E00584369105C0F0809105068111F5
:1027300014C00FE110E02EE130E044E650E0B601B5
:1027400065507109CE0144970E94B40481E08093E2
:10275000050610922D0610926A06E090DF05F090B3
:10276000E005072D9401A501B601CE010E94E30505
:10277000A8950AC08436910508F4B0CFD6CF843628
:10278000910508F4AFCFD1CFDF91CF911F910F9179
:10279000FF90EF90DF90CF90BF90AF909F908F9081
:1027A0007F900895A89580912A06813071F4A49AAB
:1027B00080E185BBA8952FEF82E597E0215080400E
:1027C0009040E1F700C0000015BAA8950895A895BB
:1027D00080912A06813021F5A49A80E185BB2FEFF4
:1027E00032E597E0215030409040E1F700C0000012
:1027F000A89515BA2FEF32E597E021503040904070
:10280000E1F700C00000A89585BB2FEF32E587E017
:10281000215030408040E1F700C00000A89515BA73
:102820000895A89580912A06813009F048C0A49A9D
:1028300080E185BBA8952FEF32E597E0215030402D
:102840009040E1F700C00000A89515BAA8952FEFB9
:1028500032E597E0215030409040E1F700C00000A1
:10286000A89585BBA8952FEF32E597E02150304021
:102870009040E1F700C00000A89515BAA8952FEF89
:1028800032E597E0215030409040E1F700C0000071
:10289000A89585BB2FEF32E587E02150304080407E
:1028A000E1F700C00000A89515BA9FEF22E537E0D8
:1028B000915020403040E1F700C00000A8950895F5
:1028C000A89510922706109219061092DA05109218
:1028D0003D061092160610920806109229061092D4
:1028E0001F06109237061092DB0585E892E00E94E1
:1028F000BE4980932A06A89586E892E00E94C649C0
:1029000090931B0680931A06A89580910C069091CF
:102910000D06892B09F055C0A895E09169068E2F08
:1029200090E08830910508F04CC0FC01EA5AFF4F56
:102930000C94A3464EE150E068E672E085EE95E027
:102940000E94AE493EC04EE150E06CE472E085EE7C
:1029500095E00E94AE4935C04EE150E060E372E080
:1029600085EE95E00E94AE492CC04EE150E064E156
:1029700072E085EE95E00E94AE4923C04EE150E042
:1029800068EF71E085EE95E00E94AE491AC04EE115
:1029900050E06CED71E085EE95E00E94AE4911C00B
:1029A0004EE150E060EC71E085EE95E00E94AE49AA
:1029B00008C04EE150E064EA71E085EE95E00E94C7
:1029C000AE49A89580910C0690910D06019719F5D6
:1029D000A89580911506813069F018F0823099F041
:1029E0001AC04EE150E068E871E085EE95E00E9483
:1029F000AE4911C04EE150E06CE671E085EE95E025
:102A00000E94AE4908C04EE150E060E571E085EEFD
:102A100095E00E94AE49A89580910C0690910D0614
:102A2000029719F5A89580911C06813069F018F07D
:102A3000823099F01AC04EE150E064E371E085EE17
:102A400095E00E94AE4911C04EE150E068E171E0AE
:102A500085EE95E00E94AE4908C04EE150E06CEF73
:102A600070E085EE95E00E94AE49A89580910C0635
:102A700090910D06049711F580917406813069F0EC
:102A800018F0823099F01AC04EE150E060EE70E02C
:102A900085EE95E00E94AE4911C04EE150E064EC35
:102AA00070E085EE95E00E94AE4908C04EE150E02E
:102AB00068EA70E085EE95E00E94AE49A8958091A5
:102AC0000C0690910D06059711F5809168068130EE
:102AD00069F018F0823099F01AC04EE150E06CE8CD
:102AE00070E085EE95E00E94AE4911C04EE150E0E5
:102AF00060E770E085EE95E00E94AE4908C04EE1C7
:102B000050E064E570E085EE95E00E94AE49A8953E
:102B100080910C0690910D06069711F5809165063F
:102B2000813069F018F0823099F01AC04EE150E01F
:102B300068E370E085EE95E00E94AE4911C04EE179
:102B400050E06CE170E085EE95E00E94AE4908C06F
:102B50004EE150E060E070E085EE95E00E94AE4905
:102B6000A89587EC90E00197F1F700C00000E5EE32
:102B7000F5E0808191819093D9058093D805828179
:102B8000938190932C0680932B068481958190935A
:102B900072068093710686819781909314068093C4
:102BA0001306808580934006828593859093120654
:102BB000809311068485958590932406809323063F
:102BC000868597859093220680932106808980933D
:102BD000D4058289938990936206809361068489E3
:102BE000958990933F0680933E0680910C069091C4
:102BF0000D06079741F48091FB059091FC05909399
:102C00000D0680930C06E5EEF5E0808D918D909396
:102C1000600680935F06828D938D9093E405809388
:102C2000E305848D958D9093070680930606A895FD
:102C300008951092760610927506BC9A80917506DA
:102C4000880F81BF1092260610922506139A809154
:102C50002506880F80938600E4DD8DE490E0909354
:102C60006C0680936B0681E090E090930B06809356
:102C70000A060895BC9A80917506880F81BF139A41
:102C800080912506880F8093860080910C06909194
:102C90000D06892B09F047C24091DF055091E005F0
:102CA0008091130690911406489F9001499F300D22
:102CB000589F300D1124ADECBCEC0E94AC469695AB
:102CC0008795969587959695879590933C068093E2
:102CD0003B0620912506309126062536310530F039
:102CE00024E630E030932606209325064091210605
:102CF000509122062091250630912606421753074F
:102D000020F4509326064093250620912706211192
:102D100014C020913806309139062233310530F441
:102D200064E670E070932606609325062333310530
:102D3000F0F121E02093270602C02130C1F5209157
:102D40002B0630912C068217930788F520913806C0
:102D5000309139062817390700F520912506309162
:102D600026062F5F3F4F4217530728F03093260661
:102D70002093250604C050932606409325062091F3
:102D80002506309126062536310588F024E630E008
:102D900030932606209325060AC0209125063091FF
:102DA00026062150310930932606209325062091CE
:102DB0002B0630912C0628173907F0F5809138063C
:102DC0009091390682179307F8F460912506709167
:102DD00026066F5F7F4F6536710528F470932606CF
:102DE0006093250606C064E670E070932606609343
:102DF000250660912506709126064617570720F490
:102E0000509326064093250628173907A8F44091C9
:102E1000250650912606821B930B0B9738F44150E0
:102E20005109509326064093250606C04B50510980
:102E30005093260640932506809140068130D9F4B0
:102E400080911906811117C0209103063091040664
:102E500080911106909112062817390761F480912C
:102E600038069091390690932C0680932B069ADCB5
:102E700081E0809319068091D405813011F580910D
:102E8000DA0581111EC080910306909104062091FD
:102E9000610630916206821B930B059790F4209196
:102EA0002B0630912C0680913E0690913F06820FB2
:102EB000931F90932C0680932B0674DC81E0809303
:102EC000DA0580913D0681111CC080910306909126
:102ED00004062091110630911206821B930B029773
:102EE00080F482E390E0909376068093750681E00B
:102EF00080933D068093080680914006811101C0B1
:102F000051DC409111065091120660916D0670914E
:102F10006E068091710690917206689F9001699F7C
:102F2000300D789F300D1124ADECBCEC0E94AC4606
:102F3000969587959695879596958795840F951F75
:102F40009093D7058093D6056091750670917606AB
:102F50006115710509F426C62091D8053091D9056F
:102F60002817390720F43093D7052093D605809190
:102F70002306909124068617970720F490937606EF
:102F800080937506809103069091040648175907AF
:102F900068F540913706411129C08217930730F533
:102FA0004091D6055091D70584179507A8F4409114
:102FB0007506509176064F5F5F4F4536510528F4F0
:102FC000509376064093750611C044E650E0509346
:102FD0007606409375060AC04091750650917606B4
:102FE00041505109509376064093750628173907CA
:102FF00088F54091750650917606821B930B0697D3
:1030000038F441505109509376064093750606C036
:103010004B50510950937606409375068091DB051D
:10302000811106C0D4DB81E080931F068093DB050D
:103030002091E1053091E20580911A0690911B06DE
:103040008217930738F4F5DD81E090E090930B064A
:1030500080930A0680911606811165C080915F06F3
:1030600090916006209111063091120628173907B9
:1030700008F059C020910306309104068217930787
:1030800089F481E080933706809329066091DD05FD
:103090007091DE054091E3055091E40564177507D2
:1030A00080F526C0409137064130E9F56091DD0595
:1030B0007091DE054091E3055091E40564177507B2
:1030C00000F528173907A0F48091750690917606CF
:1030D00001968536910528F49093760680937506BF
:1030E00010C084E690E0909376068093750609C040
:1030F000809175069091760601979093760680935D
:1031000075064617570778F41092370680916D06BA
:1031100090916E06841B950B90936E0680936D06BE
:1031200081E08093160680910C0690910D06019720
:1031300009F035C1109226061092250680913D06B1
:1031400081111BC020910306309104068091110665
:10315000909112068217930780F482E390E0909397
:1031600076068093750681E080933D06809308067D
:1031700080914006811101C015DB409111065091EC
:10318000120660916D0670916E06809171069091A5
:103190007206689F9001699F300D789F300D112451
:1031A000ADECBCEC0E94AC469695879596958795BC
:1031B00096958795840F951F9093D7058093D60594
:1031C00060917506709176066115710509F4F3C476
:1031D0002091D8053091D9052817390720F430936C
:1031E000D7052093D6058091230690912406861753
:1031F000970720F4909376068093750680910306D6
:10320000909104064817590768F540913706411117
:1032100029C08217930730F54091D6055091D70504
:1032200084179507A8F440917506509176064F5F74
:103230005F4F4536510528F4509376064093750646
:1032400011C044E650E050937606409375060AC0DC
:10325000409175065091760641505109509376067B
:10326000409375062817390788F5409175065091E7
:103270007606821B930B069738F441505109509300
:1032800076064093750606C04B505109509376065A
:10329000409375068091DB05811106C098DA81E0C4
:1032A00080931F068093DB052091E1053091E205B4
:1032B00080911A0690911B068217930738F4B9DCA7
:1032C00081E090E090930B0680930A0680911606A9
:1032D000811165C080915F06909160062091110672
:1032E000309112062817390708F059C020910306BB
:1032F000309104068217930789F481E080933706A2
:10330000809329066091DD057091DE054091E3050B
:103310005091E4056417750780F526C04091370683
:103320004130E9F56091DD057091DE054091E305DE
:103330005091E4056417750700F528173907A0F4C4
:10334000809175069091760601968536910528F450
:10335000909376068093750610C084E690E0909373
:1033600076068093750609C0809175069091760661
:10337000019790937606809375064617570778F461
:103380001092370680916D0690916E06841B950B06
:1033900090936E0680936D0681E08093160680916F
:1033A0000C0690910D06029709F01EC11092760648
:1033B0001092750680914006813009F005C4809115
:1033C0001906811101C420910306309104068091F1
:1033D0001106909112062817390709F0F5C380915C
:1033E00038069091390690932C0680932B06DAD9F3
:1033F00081E080931906E8C324E630E03093260686
:103400002093250620912106309122064091250621
:10341000509126062417350720F430932606209372
:10342000250640912706411114C04091380650915D
:1034300039064639510530F464E670E0709326068B
:103440006093250647395105F0F141E04093270686
:1034500002C04130C1F540912B0650912C068417D3
:10346000950788F540913806509139064817590755
:1034700000F540912506509126064F5F5F4F2417B7
:10348000350728F0509326064093250604C0309354
:10349000260620932506409125065091260645369E
:1034A000510588F044E650E05093260640932506E7
:1034B0000AC040912506509126064150510950936B
:1034C00026064093250640912B0650912C0648175E
:1034D000590708F089C080914006811140C0809151
:1034E00038069091390684179507F8F460912506FF
:1034F000709126066F5F7F4F6536710528F47093D3
:1035000026066093250606C064E670E070932606E2
:1035100060932506609125067091260626173707C9
:1035200020F430932606209325064817590708F003
:103530005BC02091250630912606841B950B0B97C6
:1035400038F42150310930932606209325064CC0CB
:103550002B503109309326062093250645C0813033
:1035600009F042C080910306909104064091110633
:103570005091120684179507F8F460912506709112
:1035800026066F5F7F4F6536710528F47093260617
:103590006093250606C064E670E07093260660938B
:1035A000250660912506709126062617370720F418
:1035B000309326062093250648175907A8F4209132
:1035C000250630912606841B950B0B9738F4215065
:1035D0003109309326062093250606C02B50310969
:1035E000309326062093250680910C0690910D06B7
:1035F0008430910509F0FEC04091DF055091E0054F
:103600008091130690911406489F9001499F300DB8
:10361000589F300D1124ADECBCEC0E94AC46969541
:103620008795969587959695879590933C06809378
:103630003B0620912506309126062536310530F0CF
:1036400024E630E03093260620932506409121069B
:1036500050912206209125063091260642175307E5
:1036600020F4509326064093250620912706211129
:1036700014C020913806309139062639310530F4CE
:1036800064E670E0709326066093250627393105BD
:10369000F0F121E02093270602C02130C1F52091EE
:1036A0002B0630912C068217930788F52091380657
:1036B000309139062817390700F5209125063091F9
:1036C00026062F5F3F4F4217530728F030932606F8
:1036D0002093250604C0509326064093250620918A
:1036E0002506309126062536310588F024E630E09F
:1036F00030932606209325060AC020912506309196
:103700002606215031093093260620932506209164
:103710002B0630912C0628173907F0F580913806D2
:103720009091390682179307F8F4609125067091FD
:1037300026066F5F7F4F6536710528F47093260665
:103740006093250606C064E670E0709326066093D9
:10375000250660912506709126064617570720F426
:10376000509326064093250628173907A8F4409160
:10377000250650912606821B930B0B9738F4415077
:103780005109509326064093250606C04B50510917
:1037900050932606409325068091750690917606F3
:1037A000009709F43DC24091230650912406481722
:1037B000590720F450937606409375068091380699
:1037C000909139062817390708F03FC28091750695
:1037D0009091760601968536910528F490937606A9
:1037E00080937506089584E690E090937606809322
:1037F000750608958530910509F0FEC04091DF05FA
:103800005091E0058091130690911406489F900115
:10381000499F300D589F300D1124ADECBCEC0E9437
:10382000AC469695879596958795969587959093AE
:103830003C0680933B0620912506309126062536CE
:10384000310530F024E630E030932606209325063B
:10385000409121065091220620912506309126069E
:103860004217530720F450932606409325062091D3
:103870002706211114C020913806309139062639C7
:10388000310530F464E670E07093260660932506F7
:1038900027393105F0F121E02093270602C02130BD
:1038A000C1F520912B0630912C068217930788F5DD
:1038B00020913806309139062817390700F52091F4
:1038C0002506309126062F5F3F4F4217530728F0F9
:1038D000309326062093250604C050932606409375
:1038E000250620912506309126062536310588F0DB
:1038F00024E630E030932606209325060AC0209166
:103900002506309126062150310930932606209352
:10391000250620912B0630912C0628173907F0F543
:10392000809138069091390682179307F8F46091D8
:103930002506709126066F5F7F4F6536710528F466
:10394000709326066093250606C064E670E07093C7
:103950002606609325066091250670912606461777
:10396000570720F450932606409325062817390759
:10397000A8F44091250650912606821B930B0B97C5
:1039800038F441505109509326064093250606C04D
:103990004B50510950932606409325068091750699
:1039A00090917606009709F449C140912306509101
:1039B00024064817590720F450937606409375065D
:1039C00080913806909139062817390708F03DC1D3
:1039D000809175069091760601968536910528F4BA
:1039E0009093760680937506089584E690E0909310
:1039F0007606809375060895069709F026C14091D2
:103A0000DF055091E0058091130690911406489FC0
:103A10009001499F300D589F300D1124ADECBCEC46
:103A20000E94AC469695879596958795969587952D
:103A300090933C0680933B06209125063091260604
:103A40002536310530F024E630E030932606209309
:103A5000250640912106509122062091250630919D
:103A600026064217530720F4509326064093250656
:103A700020912706211114C0209138063091390673
:103A80002639310530F464E670E0709326066093C1
:103A9000250627393105F0F121E02093270602C0E1
:103AA0002130C1F520912B0630912C068217930707
:103AB00088F520913806309139062817390700F526
:103AC00020912506309126062F5F3F4F421753075E
:103AD00028F0309326062093250604C0509326062E
:103AE000409325062091250630912606253631057E
:103AF00088F024E630E030932606209325060AC09D
:103B00002091250630912606215031093093260652
:103B10002093250620912B0630912C062817390773
:103B200008F093C080913806909139068217930768
:103B3000F8F460912506709126066F5F7F4F653619
:103B4000710528F4709326066093250606C064E686
:103B500070E07093260660932506609125067091AB
:103B600026064617570720F450932606409325064D
:103B70002817390708F069C040912506509126069C
:103B8000821B930B0B9738F4415051095093260632
:103B90004093250608954B505109509326064093B3
:103BA000250608952091D8053091D90528173907A1
:103BB00008F4D9C9E7C92091D8053091D90528174B
:103BC000390708F40CCB1ACB4091DF055091E00582
:103BD0008091130690911406489F9001499F300DE3
:103BE000589F300D1124ADECBCEC0E94AC4696956C
:103BF0008795969587959695879590933C068093A3
:103C00003B0620912506309126062536310508F41D
:103C1000F9CBF2CB80917506909176060196DECDB8
:103C200080913806909139062817390798F308953E
:103C300080917506909176060196D2CE80913806D5
:103C4000909139062817390798F3089563EC70E0CE
:103C500088E692E00E94E14962EC71E08AE692E037
:103C60000E94E14966E170E08CE692E00E94E14941
:103C700066E170E08EE692E00E94E14961E070E06A
:103C800080E792E00E94E149A8956EE670E082E745
:103C900092E00E94E14964E670E084E792E00E94CD
:103CA000E14964E670E086E792E00E94E14960E065
:103CB00070E088E792E00E94E149A89560E070E03A
:103CC0008AE792E00E94E14960E070E08CE792E0D0
:103CD0000E94E14960E070E08EE792E00E94E149D5
:103CE00060E070E080E892E00E94E14960E070E00E
:103CF00082E892E00E94E14960E070E084E892E0AE
:103D00000E94E149A89566EE70E08CE492E00E9482
:103D1000E14962EC71E08EE492E00E94E14966E1E3
:103D200070E080E592E00E94E14966E170E082E5A2
:103D300092E00E94E14961E070E084E592E00E9437
:103D4000E149A89563E770E086E592E00E94E149C9
:103D500064E670E088E592E00E94E14964E670E084
:103D60008AE592E00E94E14960E070E08CE592E033
:103D70000E94E14960E070E08EE592E00E94E14936
:103D800060E070E080E692E00E94E149A89560E082
:103D900070E082E692E00E94E14960E070E084E633
:103DA00092E00E94E14960E070E086E692E00E94C5
:103DB000E14960E070E088E692E00E94E149A89560
:103DC00063EC70E088E891E00E94E14966E170E010
:103DD0008CE891E00E94E14961E070E080E991E0C7
:103DE0000E94E1496FE070E082E991E00E94E149C0
:103DF000A89564E670E084E991E00E94E14961E001
:103E000070E08EE991E00E94E14963EC70E080EAA5
:103E100091E00E94E1496AE070E082EA91E00E944C
:103E2000E149A89562EC71E086E391E00E94E149E6
:103E300066E170E08AE391E00E94E14961E070E0B0
:103E40008CE391E00E94E1496EE670E08EE391E040
:103E50000E94E149A89564E670E082E491E00E9446
:103E6000E14962E070E08AE491E00E94E14962EC9D
:103E700071E082EE90E00E94E14966E170E084EE3C
:103E800090E00E94E14962E170E086EE90E00E94DD
:103E9000E149A89564E670E08CEE90E00E94E1496B
:103EA00064E670E08EEE90E00E94E14964E070E02C
:103EB00086EF90E00E94E1496CE271E08CEF90E0C7
:103EC0000E94E149A89562EC71E08EE890E00E94C2
:103ED000E14966E170E080E990E00E94E14966E135
:103EE00070E082E990E00E94E14961E070E084E9DD
:103EF00090E00E94E149A8956EE670E086E990E0C6
:103F00000E94E14964E670E088E990E00E94E1499E
:103F100064E670E08AE990E00E94E14965E070E0C3
:103F200082EA90E00E94E149A89562EC71E08AE3A0
:103F300090E00E94E14966E170E08EE390E00E942B
:103F4000E14961E070E080E490E00E94E1496EE6C2
:103F500070E082E490E00E94E149A89564E670E098
:103F600086E490E00E94E14966E070E08EE490E033
:103F70000E94E14963EC70E088E692E00E94E1492A
:103F8000A89508956FE070E08AE892E00E94E14908
:103F90006FE070E088E892E00E94E1496FE070E035
:103FA00086E892E00E94E14961E085E892E00E94A3
:103FB000D44961E084E892E00C94D44908958FB923
:103FC000779BFECF8FB10895CF93A39AAB9AAB980E
:103FD00080E0F5DFC82F80E0F2DFAB9A6C2F70E055
:103FE000762F6627682B687F7F777695679576951D
:103FF00067957695679580E090E00E94B24520E055
:1040000030E040E85EE30E9418460E9486457093C7
:10401000040660930306CB01CF910895CF93A79A2E
:10402000AF9AAF9880E0CBDFC82F80E0C8DFAF9AAF
:104030006C2F70E0762F6627682B687F7F777695E8
:104040006795769567957695679580E090E00E94F4
:10405000B24520E030E040E85EE30E9418460E944E
:1040600086457093390660933806CB01CF91089549
:1040700080E091E090937B0680937A06809104061D
:104080008F93809103068F938EE091E09F938F939F
:104090000E94DE468DE08A95F1F700008091E005F0
:1040A0008F938091DF058F9388E191E09F938F93A9
:1040B0000E94DE469DE09A95F1F700008091260669
:1040C0008F93809125068F9382E291E09F938F9347
:1040D0000E94DE468DE08A95F1F700008091760619
:1040E0008F93809175068F938DE291E09F938F93CC
:1040F0000E94DE469DE09A95F1F7000087E391E08B
:104100009F938F930E94DE468DE08A95F1F7000021
:10411000809139068F93809138068F938FE391E0D9
:104120009F938F930E94DE468DB79EB746960FB63B
:10413000F8949EBF0FBE8DBF80910A0690910B062A
:10414000892B41F488E491E09F938F930E94DE468F
:104150000F900F9080910A0690910B06019741F401
:104160008FE491E09F938F930E94DE460F900F9013
:104170009DE09A95F1F70000E0910C06F0910D0694
:10418000E830F10508F049C1E25AFF4F0C94A3460C
:1041900086E591E09F938F930E94DE460F900F90EB
:1041A000E09169068E2F90E08830910508F035C1C6
:1041B000FC01EA59FF4F0C94A34685E691E09F93DA
:1041C0008F930E94DE460F900F90089585E791E04F
:1041D0009F938F930E94DE460F900F90089580E882
:1041E00091E09F938F930E94DE460F900F90089569
:1041F0008FE891E09F938F930E94DE460F900F907F
:1042000008958EE991E09F938F930E94DE460F9070
:104210000F9008958DEA91E09F938F930E94DE4660
:104220000F900F9008958CEB91E09F938F930E94D5
:10423000DE460F900F9008958BEC91E09F938F9343
:104240000E94DE460F900F9008958AED91E09F93B3
:104250008F930E94DE460F900F908091150681305B
:1042600069F018F0823099F0089580E891E09F930A
:104270008F930E94DE460F900F9008958FE891E093
:104280009F938F930E94DE460F900F9008958EE9C2
:1042900091E09F938F930E94DE460F900F900895B8
:1042A0008AEE91E09F938F930E94DE460F900F90CD
:1042B00080911C06813069F018F0823099F00895E1
:1042C00080E891E09F938F930E94DE460F900F90BD
:1042D00008958FE891E09F938F930E94DE460F90A0
:1042E0000F9008958EE991E09F938F930E94DE4690
:1042F0000F900F9008958BEF91E09F938F930E9402
:10430000DE460F900F90089589E092E09F938F937F
:104310000E94DE460F900F9080917406813069F004
:1043200018F0823099F0089580E891E09F938F9380
:104330000E94DE460F900F9008958FE891E09F93C2
:104340008F930E94DE460F900F9008958EE991E0C2
:104350009F938F930E94DE460F900F9008958AE1FD
:1043600092E09F938F930E94DE460F900F90809172
:104370006806813069F018F0823099F0089580E87D
:1043800091E09F938F930E94DE460F900F900895C7
:104390008FE891E09F938F930E94DE460F900F90DD
:1043A00008958EE991E09F938F930E94DE460F90CF
:1043B0000F9008958DE292E09F938F930E94DE46C6
:1043C0000F900F9080916506813069F018F082306F
:1043D00099F0089580E891E09F938F930E94DE46C4
:1043E0000F900F9008958FE891E09F938F930E9414
:1043F000DE460F900F9008958EE991E09F938F9382
:104400000E94DE460F900F9008958FE392E09F93F5
:104410008F930E94DE460F900F900895AF92BF9247
:10442000CF92DF92EF92FF920F931F93CF93DF9380
:1044300000D000D0CDB7DEB780910A0690910B0670
:10444000019709F012C180911D0690911E06892BDB
:10445000C9F40FE110E024E230E04AE550E064E600
:1044600070E088E090E00E94B40424E230E04AE585
:1044700050E064E670E08FED90E00E94B404A895EF
:104480000E94F5070F2EF3E6CF2ED12CF02DAA2493
:10449000A394B12CE3C0A895EBDD80916B069091BD
:1044A0006C068A35910549F42FEF8DE399E421508C
:1044B00080409040E1F700C00000A89503E02FE1A4
:1044C00030E04FEF5FEF69E170E085E890E00E9437
:1044D0003613F6018081A8951C821B821A821982EC
:1044E000BE016F5F7F4FCE0103960E9418458B81FE
:1044F0009C81853C994088F089819A81883D9E40C5
:1045000060F489819A81853C994038F0B0921E060A
:10451000A0921D0610922F0645D48B819C81853C6C
:10452000994008F43FC089819A818C3D9540D0F52F
:1045300089819A81853F9140A8F1B0921E06A09290
:104540001D061092410680910C0690910D06892B54
:1045500011F40E94703680910C0690910D0601971F
:1045600011F40E94E53F80910C0690910D06029790
:1045700011F40E94074180910C0690910D0604975A
:1045800011F40E94234280910C0690910D0605972C
:1045900009F4C6D580910C0690910D06069711F48A
:1045A0000E944F3511DD0E94ED10A895FFEF21EE1E
:1045B00084E0F15020408040E1F700C000002EDD93
:1045C000A8950E947E11E0902506F090260603E053
:1045D0002FE130E04FEF5FEF6EE670E08CE190E0AE
:1045E0000E94E305E0907506F09076062FE130E03A
:1045F0004FEF5FEF6EE670E080EF90E00E94E30522
:104600000E94081380910A0690910B06892B31F5C0
:104610000E94D213A8950E946014A8950E94F507E5
:104620000FE110E024E230E04AE550E064E670E09B
:1046300088E090E00E94B40424E230E04AE550E0D3
:1046400064E670E08FED90E00E94B4041092E00503
:104650001092DF0510921E0610921D0680910A0628
:1046600090910B06019709F416CF0F900F900F90C1
:104670000F90DF91CF911F910F91FF90EF90DF90FE
:10468000CF90BF90AF900895EF92FF920F931F933A
:10469000CF93DF9380912E06813009F07CC18FE1AA
:1046A00090E00E941D060E94CB0C85E080933406AA
:1046B00080912E06813009F06EC1C1E0D5E00E94E4
:1046C000070E809134068230D9F480915E068F5FA8
:1046D00080935E060FE110E02CE330E046EE50E000
:1046E00069E670E081E090E00E94B40422E330E0EB
:1046F00043EC50E068E270E088E090E00E94B4048F
:10470000809134068330D9F480915E068150809385
:104710005E060FE110E02CE330E046EE50E069E683
:1047200070E081E090E00E94B40422E330E043ECCA
:1047300050E068E270E088E090E00E94B40480916C
:104740005E06853018F010925E0610C0823009F4C3
:1047500051C028F4882351F0813051F1EEC08330EC
:1047600009F46AC0843009F4A9C0E7C00F2EF9E942
:10477000EF2EF5E0FF2EF02D0C2F2FE130E04FEF64
:104780005FEF6CE370E08FE090E00E9493058AE8B1
:1047900092E00E94C6497C0103E02FE130E04FEF38
:1047A0005FEF62E870E080E590E00E94E305C5C03D
:1047B0000F2EF0E8EF2EF5E0FF2EF02D0C2F2FE15D
:1047C00030E04FEF5FEF6CE370E088E090E00E9434
:1047D000930588E892E00E94C6497C0103E02FE13E
:1047E00030E04FEF5FEF62E870E080E590E00E941C
:1047F000E305A3C00F2EF4E7EF2EF5E0FF2EF02D1A
:104800000C2F2FE130E04FEF5FEF6CE370E082E3BD
:1048100090E00E94930586E892E00E94C6497C01E0
:1048200003E02FE130E04FEF5FEF62E870E080E5FA
:1048300090E00E94E30581C00F2EFCE5EF2EF5E02D
:10484000FF2EF02D0C2F2FE130E04FEF5FEF6CE3E8
:1048500070E088E290E00E9493050F2EFAE6EF2EBA
:10486000F5E0FF2EF02D02E02FE130E04FEF5FEF9B
:1048700062E870E088E290E00E949305809134063F
:10488000811179C0E3D97EDB0F2EF6E2EF2EF5E041
:10489000FF2EF02D2FE130E04FEF5FEF62E870E088
:1048A00088E290E00E9493052FEF89E698E121507D
:1048B00080409040E1F700C000005DC00F2EFBE497
:1048C000EF2EF5E0FF2EF02D0C2F2FE130E04FEF13
:1048D0005FEF6CE370E08EE190E00E94930585E865
:1048E00092E00E94BE49813089F40F2EFDE3EF2E45
:1048F000F5E0FF2EF02D03E02FE130E04FEF5FEF0A
:1049000062E870E080E590E00E94930585E892E01F
:104910000E94BE49811111C00F2EF8E3EF2EF5E081
:10492000FF2EF02D03E02FE130E04FEF5FEF62E864
:1049300070E080E590E00E9493058091340681301C
:1049400089F410922E0610921E0610921D068FE119
:1049500090E00E941D0681E090E090930B0680930A
:104960000A065CDD80913406811105C0C0932E06D5
:104970001092700617D0D09334062FE785EB91E0A4
:10498000215080409040E1F700C0000080912E0649
:10499000813009F494CEDF91CF911F910F91FF9058
:1049A000EF900895AF92BF92CF92DF92EF92FF9275
:1049B0000F931F93CF93DF93809170068111E7C10E
:1049C00085E0809334060F2EF9E1CF2ED12CF02D07
:1049D0000F2EF5E0AF2EB12CF02DD1E0C5E0809187
:1049E0005E06813009F478C038F0823009F4E4C002
:1049F000843009F451C1B7C18AE892E00E94C649E7
:104A00007C0103E02FE130E040E058EF62E870E025
:104A100080E590E00E94E3058AE892E00E94C649A2
:104A200090933306809332060E94070E80913406DD
:104A30008230A9F4809132069091330601969093CA
:104A40003306809332060FE110E02CE330E046EEAF
:104A500050E069E670E081E090E00E94B40480914B
:104A600034068330A9F48091320690913306019781
:104A700090933306809332060FE110E02CE330E090
:104A800046EE50E069E670E081E090E00E94B404F8
:104A900080913206909133068A31910528F0D092A8
:104AA0003306C092320606C00A9720F4D09233062D
:104AB000C092320660913206709133068AE892E025
:104AC0000E94E1492FE788E391E021508040904027
:104AD000E1F700C0000047C188E892E00E94C649A3
:104AE0007C0103E02FE130E040E058EF62E870E045
:104AF00080E590E00E94E30588E892E00E94C649C4
:104B00009093100680930F060E94070E8091340642
:104B10008230A9F480910F0690911006019690932F
:104B2000100680930F060FE110E02CE330E046EE14
:104B300050E069E670E081E090E00E94B40480916A
:104B400034068330A9F480910F06909110060197E6
:104B50009093100680930F060FE110E02CE330E0F5
:104B600046EE50E069E670E081E090E00E94B40417
:104B700080910F06909110068A31910528F0D0920D
:104B80001006C0920F0606C00A9720F4D0921006B5
:104B9000C0920F0660910F067091100688E892E0AF
:104BA0000E94E1492FE788E391E021508040904046
:104BB000E1F700C00000D7C086E892E00E94C64935
:104BC0007C0103E02FE130E040E058EF62E870E064
:104BD00080E590E00E94E30586E892E00E94C649E5
:104BE00090933106809330060E94070E8091340620
:104BF0008230A9F48091300690913106019690930D
:104C00003106809330060FE110E02CE330E046EEF1
:104C100050E069E670E081E090E00E94B404809189
:104C200034068330A9F480913006909131060197C3
:104C300090933106809330060FE110E02CE330E0D2
:104C400046EE50E069E670E081E090E00E94B40436
:104C500080913006909131068F31910528F0B09205
:104C60003106A092300606C0059720F4B0923106B6
:104C7000A0923006609130067091310686E892E08D
:104C80000E94E1492FE788E391E021508040904065
:104C9000E1F700C0000067C085E892E00E94BE49CD
:104CA0008093D5050E94070E80913406823089F4E6
:104CB0008091D5058F5F8093D5050FE110E02CE33F
:104CC00030E046EE50E069E670E081E090E00E945E
:104CD000B40480913406833089F48091D5058150E5
:104CE0008093D5050FE110E02CE330E046EE50E074
:104CF00069E670E081E090E00E94B4048091D505FF
:104D0000823018F01092D50517C0813089F40F2E2B
:104D1000FDE3EF2EF5E0FF2EF02D03E02FE130E074
:104D200040E058EF62E870E080E590E00E94930573
:104D30008091D505811111C00F2EF8E3EF2EF5E01B
:104D4000FF2EF02D03E02FE130E040E058EF62E865
:104D500070E080E590E00E9493056091D50585E8BC
:104D600092E00E94D44980913406813049F4D09376
:104D70007006D0932E068FE190E00E941D0684DC21
:104D8000C093340680917006882309F428CEDF9101
:104D9000CF911F910F91FF90EF90DF90CF90BF9038
:104DA000AF9008952F923F924F925F926F927F92B1
:104DB0008F929F92AF92BF92CF92DF92EF92FF922B
:104DC0000F931F93CF93DF9380912F06811195C18D
:104DD0008FE190E00E941D060E942F0C85E08093D9
:104DE000340610922E061092280680912F0681110B
:104DF00084C122242394C5EED5E00F2EF7E06F2E58
:104E0000712CF02D0F2EF6E08F2E912CF02D0F2E01
:104E1000F5E0AF2EB12CF02D6894CC24C2F8D12C43
:104E20000F2EF3E04F2E512CF02D0F2EF5E03F2EDC
:104E3000F02D0E94070E80913406823089F4809113
:104E400028068F5F809328060FE110E02CE330E006
:104E500046EE50E069E670E081E090E00E94B40424
:104E600080913406833089F48091280681508093A4
:104E700028060FE110E02CE330E046EE50E069E652
:104E800070E081E090E00E94B404E0912806E930EF
:104E900018F0109228060BC08E2F90E089309105F3
:104EA00008F0F1C0FC01E259FF4F0C94A3460F2E0D
:104EB000F8E0EF2EF5E0FF2EF02D02E02FE130E0DC
:104EC0004FEF5FEF62E870E088E090E00E949305AA
:104ED00010922E0610920D0610920C0609C10F2E8C
:104EE000FAEFEF2EF4E0FF2EF02D02E02FE130E09C
:104EF0004FEF5FEF68E770E088E090E00E94930575
:104F000010922E0681E090E090930D0680930C069F
:104F1000EFC00F2EFCEEEF2EF4E0FF2EF02D02E09E
:104F20002FE130E04FEF5FEF68E770E088E090E05E
:104F30000E94930510922E0682E090E090930D0659
:104F400080930C06D5C00F2EF0EEEF2EF4E0FF2E6E
:104F5000F02D02E02FE130E04FEF5FEF68E770E007
:104F600088E090E00E94930510922E0650920D0664
:104F700040920C06BDC00F2EFEECEF2EF4E0FF2E8B
:104F8000F02D02E02FE130E04FEF5FEF68E770E0D7
:104F900088E090E00E94930510922E06D0920D06B4
:104FA000C0920C06A5C00F2EF8ECEF2EF4E0FF2EF9
:104FB000F02D02E02FE130E04FEF5FEF6EE670E0A2
:104FC00088E290E00E9493050F2EFEEBEF2EF4E0B6
:104FD000FF2EF02D2FE130E04FEF5FEF67E870E03C
:104FE0008FE090E00E94930510922E06B0920D067D
:104FF000A0920C067DC00F2EF1EBEF2EF4E0FF2EF9
:10500000F02D02E02FE130E04FEF5FEF68E770E056
:1050100088E090E00E94930510922E0690920D0673
:1050200080920C0665C00F2EF3E9EF2EF4E0FF2E00
:10503000F02D02E02FE130E04FEF5FEF68E770E026
:1050400088E090E00E94930510922E0670920D0663
:1050500060920C064DC00F2EFDE9EF2EF4E0FF2EFE
:10506000F02D02E02FE130E04FEF5FEF68E770E0F6
:1050700082E090E00E94930520922E0680913406F3
:10508000813029F508C080913406813001F5809186
:105090002E06813059F410920D0610920C061092D3
:1050A0002F068FE190E00E941D06EEDA20922F0677
:1050B00010921E0610921D0680910C0690910D060E
:1050C0009F8B8E8B8FE190E00E941D06A7D93092B6
:1050D00034062FEF80E792E0215080409040E1F7C6
:1050E00000C0000080912F06882309F4A2CE05C0DD
:1050F00080913406813059F7D9CFDF91CF911F913C
:105100000F91FF90EF90DF90CF90BF90AF909F9066
:105110008F907F906F905F904F903F902F90089569
:10512000EF92FF920F931F93CF93DF93A8958091F7
:10513000410681110DC18FE190E00E941D060E9481
:10514000680D8091680690E090931806809317068A
:1051500085E080933406809141068111F9C0C1E059
:10516000D5E0A8950E94070E809134068230A9F4FC
:1051700080911706909118060196909318068093D7
:1051800017060FE110E02CE330E046EE50E069E650
:1051900070E081E090E00E94B40480913406833096
:1051A000A9F480911706909118060197909318061C
:1051B000809317060FE110E02CE330E046EE50E05C
:1051C00069E670E081E090E00E94B40480911706E7
:1051D000909118068330910528F0109218061092CD
:1051E000170607C08130910501F118F00297C9F147
:1051F00054C00F2EFFE7EF2EF4E0FF2EF02D02E05B
:105200002FE130E04FEF5FEF6DE770E088E290E074
:105210000E949305109268064EE150E06CE870E041
:1052200085EE95E00E94AE4938C00F2EF5E7EF2ECF
:10523000F4E0FF2EF02D02E02FE130E04FEF5FEFC2
:105240006DE770E088E290E00E949305C0936806E5
:105250004EE150E060E770E085EE95E00E94AE49D7
:105260001CC00F2EFBE6EF2EF4E0FF2EF02D02E027
:105270002FE130E04FEF5FEF6DE770E088E290E004
:105280000E94930582E0809368064EE150E064E559
:1052900070E085EE95E00E94AE4980913406811160
:1052A0000FC0A895C093410610921E0610921D06CD
:1052B000C0932F068FE190E00E941D06A895AED8FE
:1052C000809134068130A1F5A895C09341061092D3
:1052D0001E0610921D06C0932F068FE190E00E94DB
:1052E0001D06A8951092770680916806813069F0B6
:1052F00018F0823099F01AC04EE150E06CE870E08E
:1053000085EE95E00E94AE4911C04EE150E060E7A5
:1053100070E085EE95E00E94AE4908C04EE150E095
:1053200064E570E085EE95E00E94AE49A89517D03F
:10533000D09334062FEF80E792E0215080409040D8
:10534000E1F700C0000080914106882309F409CFED
:10535000DF91CF911F910F91FF90EF900895DF9211
:10536000EF92FF920F931F93CF93DF938091770675
:1053700081110C9447358FE190E00E941D060E9438
:105380006F0E85E0809334068091770681110C942E
:105390004735C5EED5E00F2EF5E0DF2EF02D0E944B
:1053A000070E809134068230D9F4809163068F5FB6
:1053B000809363060FE110E02CE330E046EE50E00E
:1053C00069E670E081E090E00E94B40422E330E0FE
:1053D00043EC50E068E270E088E090E00E94B404A2
:1053E000809134068330D9F4809163068150809394
:1053F00063060FE110E02CE330E046EE50E069E692
:1054000070E081E090E00E94B40422E330E043ECDD
:1054100050E068E270E088E090E00E94B404E0911F
:105420006306EE3018F0109263060CC08E2F90E0E9
:105430008E30910510F00C94C833FC01E958FF4FF1
:105440000C94A34680910C0690910D06892B71F562
:105450000F2EF5E2EF2EF4E0FF2EF02D01E02FE10C
:1054600030E04FEF5FEF62E370E08FE090E00E948A
:1054700093050F2EFEE1EF2EF4E0FF2EF02D2FE12D
:1054800030E04FEF5FEF66E470E08CE390E00E9465
:105490009305E880F98003E02FE130E04FEF5FEF04
:1054A00062E870E080E590E00E94E30580910C06E0
:1054B00090910D06019771F50F2EF5E2EF2EF4E0B5
:1054C000FF2EF02D01E02FE130E04FEF5FEF62E3C0
:1054D00070E08FE090E00E9493050F2EFEE1EF2E2A
:1054E000F4E0FF2EF02D2FE130E04FEF5FEF66E4A8
:1054F00070E08CE390E00E949305E880F98003E07F
:105500002FE130E04FEF5FEF62E870E080E590E080
:105510000E94E30580910C0690910D068230910562
:1055200031F4209163062F5F2093630614C084300A
:10553000910539F4809163068F5F809363060C9424
:10554000C8338530910539F4809163068F5F80936D
:1055500063060C94C833069711F00C94C8338091FD
:1055600063068F5F809363060C94C83380910C06AA
:1055700090910D06892B71F50F2EF6E0EF2EF4E0D9
:10558000FF2EF02D01E02FE130E04FEF5FEF62E3FF
:1055900070E08FE090E00E9493050F2EF8EFEF2E61
:1055A000F3E0FF2EF02D2FE130E04FEF5FEF66E4E8
:1055B00070E08CE390E00E949305EA80FB8003E0BA
:1055C0002FE130E04FEF5FEF62E870E080E590E0C0
:1055D0000E94E30580910C0690910D0681309105A3
:1055E00031F4809163068F5F8093630664C00297F5
:1055F00071F50F2EF6E0EF2EF4E0FF2EF02D01E016
:105600002FE130E04FEF5FEF62E370E08FE090E07A
:105610000E9493050F2EF8EFEF2EF3E0FF2EF02DF2
:105620002FE130E04FEF5FEF66E470E08CE390E055
:105630000E949305EA80FB8003E02FE130E04FEF0A
:105640005FEF62E870E080E590E00E94E305809102
:105650000C0690910D06049771F50F2EF6E0EF2ED3
:10566000F4E0FF2EF02D01E02FE130E04FEF5FEF8F
:1056700062E370E08FE090E00E9493050F2EF8EF58
:10568000EF2EF3E0FF2EF02D2FE130E04FEF5FEF34
:1056900066E470E08CE390E00E949305EA80FB8072
:1056A00003E02FE130E04FEF5FEF62E870E080E56C
:1056B00090E00E94E30580910C0690910D060597FD
:1056C00071F50F2EF6E0EF2EF4E0FF2EF02D01E045
:1056D0002FE130E04FEF5FEF62E370E08FE090E0AA
:1056E0000E9493050F2EF8EFEF2EF3E0FF2EF02D22
:1056F0002FE130E04FEF5FEF66E470E08CE390E085
:105700000E949305EA80FB8003E02FE130E04FEF39
:105710005FEF62E870E080E590E00E94E305809131
:105720000C0690910D06069711F00C94C8330F2EBD
:10573000F6E0EF2EF4E0FF2EF02D01E02FE130E057
:105740004FEF5FEF62E370E08FE090E00E9493051F
:105750000F2EF8EFEF2EF3E0FF2EF02D2FE130E0CB
:105760004FEF5FEF66E470E08CE390E00E949305FA
:10577000EA80FB8003E02FE130E04FEF5FEF62E86B
:1057800070E080E590E00E94E3050C94C8338091BE
:105790000C0690910D06892B71F50F2EF0EEEF2E71
:1057A000F3E0FF2EF02D01E02FE130E04FEF5FEF4F
:1057B00062E370E08FE090E00E9493050F2EF8EC1A
:1057C000EF2EF3E0FF2EF02D2FE130E04FEF5FEFF3
:1057D00066E470E08FE090E00E949305EC80FD802D
:1057E00003E02FE130E04FEF5FEF62E870E080E52B
:1057F00090E00E94E30580910C0690910D060197C0
:1058000071F50F2EF0EEEF2EF3E0FF2EF02D01E0FC
:105810002FE130E04FEF5FEF62E370E08FE090E068
:105820000E9493050F2EF8ECEF2EF3E0FF2EF02DE3
:105830002FE130E04FEF5FEF66E470E08FE090E043
:105840000E949305EC80FD8003E02FE130E04FEFF4
:105850005FEF62E870E080E590E00E94E3058091F0
:105860000C0690910D068230910531F4209163066B
:105870002F5F2093630612C08430910531F480912C
:1058800063068F5F8093630683C78530910531F48B
:10589000809163068F5F809363067AC7069709F04D
:1058A00077C7809163068F5F8093630671C780918D
:1058B0000C0690910D06892B71F50F2EF0EBEF2E53
:1058C000F3E0FF2EF02D01E02FE130E04FEF5FEF2E
:1058D00062E370E08FE090E00E9493050F2EF8E9FC
:1058E000EF2EF3E0FF2EF02D2FE130E04FEF5FEFD2
:1058F00066E470E08FE090E00E949305EE80FF8008
:1059000003E02FE130E04FEF5FEF62E870E080E509
:1059100090E00E94E30580910C0690910D06813085
:10592000910531F4809163068F5F8093630664C0B4
:10593000029771F50F2EF0EBEF2EF3E0FF2EF02D16
:1059400001E02FE130E04FEF5FEF62E370E08FE0C6
:1059500090E00E9493050F2EF8E9EF2EF3E0FF2E62
:10596000F02D2FE130E04FEF5FEF66E470E08FE065
:1059700090E00E949305EE80FF8003E02FE130E08D
:105980004FEF5FEF62E870E080E590E00E94E30592
:1059900080910C0690910D06049771F50F2EF0EB97
:1059A000EF2EF3E0FF2EF02D01E02FE130E04FEF7E
:1059B0005FEF62E370E08FE090E00E9493050F2EAE
:1059C000F8E9EF2EF3E0FF2EF02D2FE130E04FEF5E
:1059D0005FEF66E470E08FE090E00E949305EE8058
:1059E000FF8003E02FE130E04FEF5FEF62E870E00F
:1059F00080E590E00E94E30580910C0690910D06F1
:105A0000059771F50F2EF0EBEF2EF3E0FF2EF02D42
:105A100001E02FE130E04FEF5FEF62E370E08FE0F5
:105A200090E00E9493050F2EF8E9EF2EF3E0FF2E91
:105A3000F02D2FE130E04FEF5FEF66E470E08FE094
:105A400090E00E949305EE80FF8003E02FE130E0BC
:105A50004FEF5FEF62E870E080E590E00E94E305C1
:105A600080910C0690910D06069709F091C60F2EB5
:105A7000F0EBEF2EF3E0FF2EF02D01E02FE130E010
:105A80004FEF5FEF62E370E08FE090E00E949305DC
:105A90000F2EF8E9EF2EF3E0FF2EF02D2FE130E08E
:105AA0004FEF5FEF66E470E08FE090E00E949305B7
:105AB000EE80FF8003E02FE130E04FEF5FEF62E820
:105AC00070E080E590E00E94E30562C680910C06DC
:105AD00090910D06892BD9F50F2EF0E8EF2EF3E00B
:105AE000FF2EF02D01E02FE130E04FEF5FEF6CE390
:105AF00070E08FE090E00E9493058885998501977A
:105B000089F40F2EFDE3EF2EF5E0FF2EF02D03E0DC
:105B10002FE130E04FEF5FEF62E870E080E590E06A
:105B20000E94930588859985892B89F40F2EF8E3C7
:105B3000EF2EF5E0FF2EF02D03E02FE130E04FEFE8
:105B40005FEF62E870E080E590E00E94930580914D
:105B50000C0690910D060197D9F50F2EF0E8EF2E67
:105B6000F3E0FF2EF02D01E02FE130E04FEF5FEF8B
:105B70006CE370E08FE090E00E9493058885998542
:105B8000019789F40F2EFDE3EF2EF5E0FF2EF02DA7
:105B900003E02FE130E04FEF5FEF62E870E080E577
:105BA00090E00E94930588859985892B89F40F2EB2
:105BB000F8E3EF2EF5E0FF2EF02D03E02FE130E0CB
:105BC0004FEF5FEF62E870E080E590E00E949305A0
:105BD00080910C0690910D060297D9F50F2EF0E8F2
:105BE000EF2EF3E0FF2EF02D01E02FE130E04FEF3C
:105BF0005FEF6CE370E08FE090E00E949305888592
:105C00009985019789F40F2EFDE3EF2EF5E0FF2E25
:105C1000F02D03E02FE130E04FEF5FEF62E870E03E
:105C200080E590E00E94930588859985892B89F409
:105C30000F2EF8E3EF2EF5E0FF2EF02D03E02FE11D
:105C400030E04FEF5FEF62E870E080E590E00E94A7
:105C5000930580910C0690910D068430910531F4E6
:105C6000809163068F5F8093630692C585309105AE
:105C700031F4809163068F5F8093630689C5069730
:105C800009F086C50F2EF0E8EF2EF3E0FF2EF02D81
:105C900001E02FE130E04FEF5FEF6CE370E08FE069
:105CA00090E00E94930588859985019789F40F2ECD
:105CB000FDE3EF2EF5E0FF2EF02D03E02FE130E0C5
:105CC0004FEF5FEF62E870E080E590E00E9493059F
:105CD00088859985892B09F05BC50F2EF8E3EF2E97
:105CE000F5E0FF2EF02D03E02FE130E04FEF5FEF06
:105CF00062E870E080E590E00E94930549C58091DC
:105D00000C0690910D06892B71F50F2EF8E6EF2EFB
:105D1000F3E0FF2EF02D01E02FE130E04FEF5FEFD9
:105D200062E370E08FE090E00E9493050F2EF0E5B3
:105D3000EF2EF3E0FF2EF02D2FE130E04FEF5FEF7D
:105D400066E470E08FE090E00E949305EA84FB84B3
:105D500003E02FE130E04FEF5FEF62E870E080E5B5
:105D600090E00E94E30580910C0690910D0601974A
:105D700071F50F2EF8E6EF2EF3E0FF2EF02D01E087
:105D80002FE130E04FEF5FEF62E370E08FE090E0F3
:105D90000E9493050F2EF0E5EF2EF3E0FF2EF02D7D
:105DA0002FE130E04FEF5FEF66E470E08FE090E0CE
:105DB0000E949305EA84FB8403E02FE130E04FEF7B
:105DC0005FEF62E870E080E590E00E94E30580917B
:105DD0000C0690910D06029771F50F2EF8E6EF2E46
:105DE000F3E0FF2EF02D01E02FE130E04FEF5FEF09
:105DF00062E370E08FE090E00E9493050F2EF0E5E3
:105E0000EF2EF3E0FF2EF02D2FE130E04FEF5FEFAC
:105E100066E470E08FE090E00E949305EA84FB84E2
:105E200003E02FE130E04FEF5FEF62E870E080E5E4
:105E300090E00E94E30580910C0690910D0684305D
:105E4000910531F4809163068F5F80936306A0C44F
:105E50008530910531F4809163068F5F80936306EE
:105E600097C4069709F094C40F2EF8E6EF2EF3E0DE
:105E7000FF2EF02D01E02FE130E04FEF5FEF62E306
:105E800070E08FE090E00E9493050F2EF0E5EF2E7A
:105E9000F3E0FF2EF02D2FE130E04FEF5FEF66E4EF
:105EA00070E08FE090E00E949305EA84FB8403E0B9
:105EB0002FE130E04FEF5FEF62E870E080E590E0C7
:105EC0000E94E30565C480910C0690910D06892B14
:105ED00071F50F2EF8E3EF2EF3E0FF2EF02D01E029
:105EE0002FE130E04FEF5FEF62E370E08FE090E092
:105EF0000E9493050F2EF0E2EF2EF3E0FF2EF02D1F
:105F00002FE130E04FEF5FEF66E470E08FE090E06C
:105F10000E949305EC84FD8403E02FE130E04FEF15
:105F20005FEF62E870E080E590E00E94E305809119
:105F30000C0690910D06019771F50F2EF8E3EF2EE8
:105F4000F3E0FF2EF02D01E02FE130E04FEF5FEFA7
:105F500062E370E08FE090E00E9493050F2EF0E284
:105F6000EF2EF3E0FF2EF02D2FE130E04FEF5FEF4B
:105F700066E470E08FE090E00E949305EC84FD847D
:105F800003E02FE130E04FEF5FEF62E870E080E583
:105F900090E00E94E30580910C0690910D068230FE
:105FA000910531F4809163068F5F8093630664C02E
:105FB000049771F50F2EF8E3EF2EF3E0FF2EF02D8E
:105FC00001E02FE130E04FEF5FEF62E370E08FE040
:105FD00090E00E9493050F2EF0E2EF2EF3E0FF2EEB
:105FE000F02D2FE130E04FEF5FEF66E470E08FE0DF
:105FF00090E00E949305EC84FD8403E02FE130E003
:106000004FEF5FEF62E870E080E590E00E94E3050B
:1060100080910C0690910D06059771F50F2EF8E30F
:10602000EF2EF3E0FF2EF02D01E02FE130E04FEFF7
:106030005FEF62E370E08FE090E00E9493050F2E27
:10604000F0E2EF2EF3E0FF2EF02D2FE130E04FEFE6
:106050005FEF66E470E08FE090E00E949305EC84CF
:10606000FD8403E02FE130E04FEF5FEF62E870E086
:1060700080E590E00E94E30580910C0690910D066A
:10608000069709F085C3809163068F5F809363064E
:106090007FC380910C0690910D06892B71F50F2E10
:1060A000F8E0EF2EF3E0FF2EF02D01E02FE130E0DD
:1060B0004FEF5FEF62E370E08FE090E00E949305A6
:1060C0000F2EF0EFEF2EF2E0FF2EF02D2FE130E05B
:1060D0004FEF5FEF66E470E08FE090E00E94930581
:1060E000EE84FF8403E02FE130E04FEF5FEF62E8E2
:1060F00070E080E590E00E94E30580910C069091AD
:106100000D068130910531F4809163068F5F809395
:10611000630664C0029771F50F2EF8E0EF2EF3E0EE
:10612000FF2EF02D01E02FE130E04FEF5FEF62E353
:1061300070E08FE090E00E9493050F2EF0EFEF2EBD
:10614000F2E0FF2EF02D2FE130E04FEF5FEF66E43D
:1061500070E08FE090E00E949305EE84FF8403E0FE
:106160002FE130E04FEF5FEF62E870E080E590E014
:106170000E94E30580910C0690910D06049771F53D
:106180000F2EF8E0EF2EF3E0FF2EF02D01E02FE1CF
:1061900030E04FEF5FEF62E370E08FE090E00E944D
:1061A00093050F2EF0EFEF2EF2E0FF2EF02D2FE1F2
:1061B00030E04FEF5FEF66E470E08FE090E00E9428
:1061C0009305EE84FF8403E02FE130E04FEF5FEFB3
:1061D00062E870E080E590E00E94E30580910C06A3
:1061E00090910D06059771F50F2EF8E0EF2EF3E074
:1061F000FF2EF02D01E02FE130E04FEF5FEF62E383
:1062000070E08FE090E00E9493050F2EF0EFEF2EEC
:10621000F2E0FF2EF02D2FE130E04FEF5FEF66E46C
:1062200070E08FE090E00E949305EE84FF8403E02D
:106230002FE130E04FEF5FEF62E870E080E590E043
:106240000E94E30580910C0690910D06069709F0D7
:106250009FC20F2EF8E0EF2EF3E0FF2EF02D01E0AD
:106260002FE130E04FEF5FEF62E370E08FE090E00E
:106270000E9493050F2EF0EFEF2EF2E0FF2EF02D8F
:106280002FE130E04FEF5FEF66E470E08FE090E0E9
:106290000E949305EE84FF8403E02FE130E04FEF8E
:1062A0005FEF62E870E080E590E00E94E30570C275
:1062B00080910C0690910D06892BF1F40F2EF0E7DA
:1062C000EF2EF2E0FF2EF02D01E02FE130E04FEF56
:1062D0005FEF6CE370E08FE090E00E949305E88C44
:1062E000F98C03E02FE130E04FEF5FEF62E870E000
:1062F00080E590E00E94E30580910C0690910D06E8
:106300000197F1F40F2EF0E7EF2EF2E0FF2EF02DC3
:1063100001E02FE130E04FEF5FEF6CE370E08FE0E2
:1063200090E00E949305E88CF98C03E02FE130E0C7
:106330004FEF5FEF62E870E080E590E00E94E305D8
:1063400080910C0690910D068230910531F42091D8
:1063500063062F5F2093630612C08430910531F4E9
:10636000809163068F5F8093630612C2853091052A
:1063700031F4809163068F5F8093630609C20697AC
:1063800009F006C2809163068F5F8093630600C2A6
:1063900080910C0690910D06892BF1F40F2EF6ECEE
:1063A000EF2EF2E0FF2EF02D01E02FE130E04FEF75
:1063B0005FEF6CE370E08FE090E00E949305EA8C61
:1063C000FB8C03E02FE130E04FEF5FEF62E870E01D
:1063D00080E590E00E94E30580910C0690910D0607
:1063E0000197F1F40F2EF6ECEF2EF2E0FF2EF02DD8
:1063F00001E02FE130E04FEF5FEF6CE370E08FE002
:1064000090E00E949305EA8CFB8C03E02FE130E0E2
:106410004FEF5FEF62E870E080E590E00E94E305F7
:1064200080910C0690910D068230910531F42091F7
:1064300063062F5F2093630612C08430910531F408
:10644000809163068F5F80936306A2C185309105BA
:1064500031F4809163068F5F8093630699C106973C
:1064600009F096C1809163068F5F8093630690C1A7
:1064700080910C0690910D06892BF1F50F2EFEED03
:10648000EF2EF2E0FF2EF02D01E02FE130E04FEF94
:106490005FEF6CE370E08EE190E00E9493058889E5
:1064A0009989019789F40F2EFDE3EF2EF5E0FF2E79
:1064B000F02D03E02FE130E04FEF5FEF62E870E096
:1064C00080E590E00E94930588899989892B89F459
:1064D0000F2EF8E3EF2EF5E0FF2EF02D03E02FE175
:1064E00030E04FEF5FEF62E870E080E590E00E94FF
:1064F000930588898093D40580910C0690910D06B0
:106500008130910531F4209163062F5F209363065B
:1065100012C08230910531F4209163062F5F2093E1
:10652000630612C08430910531F4809163068F5F59
:10653000809363062DC18530910531F48091630607
:106540008F5F8093630624C1069709F021C1809173
:1065500063068F5F809363061BC180910C06909148
:106560000D060097A9F52091D405211188C210923B
:10657000630644C00F2EF8E6EF2EF3E0FF2EF02D59
:1065800001E02FE130E04FEF5FEF62E370E08FE07A
:1065900090E00E9493050F2EF0EBEF2EF2E0FF2E1D
:1065A000F02D2FE130E04FEF5FEF66E470E08FE019
:1065B00090E00E949305EA88FB8803E02FE130E039
:1065C0004FEF5FEF62E870E080E590E00E94E30546
:1065D00080910C0690910D068130910531F4209147
:1065E00063062F5F2093630612C08230910531F459
:1065F000209163062F5F2093630612C084309105BB
:1066000031F4809163068F5F80936306C1C085304B
:10661000910531F4809163068F5F80936306B8C063
:10662000069709F0B5C0809163068F5F809363067B
:10663000AFC080910C0690910D060097A9F52091AE
:10664000D405211120C21092630644C00F2EF9E92F
:10665000EF2EF2E0FF2EF02D01E02FE130E04FEFC2
:106660005FEF62E370E08FE090E00E9493050F2EF1
:10667000F6E8EF2EF2E0FF2EF02D2FE130E04FEFA5
:106680005FEF66E470E08FE090E00E949305EC8895
:10669000FD8803E02FE130E04FEF5FEF62E870E04C
:1066A00080E590E00E94E30580910C0690910D0634
:1066B0008130910531F4209163062F5F20936306AA
:1066C00012C08230910531F4209163062F5F209330
:1066D000630612C08430910531F4809163068F5FA8
:1066E0008093630655C08530910531F4809163062F
:1066F0008F5F809363064CC0069709F049C0809174
:1067000063068F5F8093630643C080910C0690916F
:106710000D06009719F4109263060CC081309105A4
:1067200019F41092630626C08230910519F4109274
:1067300063062EC00497F1F40F2EF9E4EF2EF2E079
:10674000FF2EF02D01E02FE130E04FEF5FEF6CE323
:1067500070E08FE090E00E949305EC8CFD8C03E0EC
:106760002FE130E04FEF5FEF62E870E080E590E00E
:106770000E94E30580910C0690910D0685309105ED
:1067800019F41092630604C0069711F41092630680
:1067900080913406813009F050C1809377061092C1
:1067A000410680910C0690910D06892B09F04BC093
:1067B000E0911706F0911806E830F10508F043C0A3
:1067C000EB57FF4F0C94A3464EE150E068E672E0B1
:1067D000CE010E94CB4937C04EE150E06CE472E03C
:1067E000CE010E94CB492FC04EE150E060E372E041
:1067F000CE010E94CB4927C04EE150E064E172E037
:10680000CE010E94CB491FC04EE150E068EF71E01D
:10681000CE010E94CB4917C04EE150E06CED71E013
:10682000CE010E94CB490FC04EE150E060EC71E018
:10683000CE010E94CB4907C04EE150E064EA71E00E
:10684000CE010E94CB4980910C0690910D060197D4
:1068500011F580911706909118068130910561F02D
:1068600018F0029789F017C04EE150E068E871E037
:10687000CE010E94CB490FC04EE150E06CE671E0C2
:10688000CE010E94CB4907C04EE150E060E571E0C7
:10689000CE010E94CB4980910C0690910D06029783
:1068A00011F580911706909118068130910561F0DD
:1068B00018F0029789F017C04EE150E064E371E0F0
:1068C000CE010E94CB490FC04EE150E068E171E07B
:1068D000CE010E94CB4907C04EE150E06CEF70E062
:1068E000CE010E94CB4980910C0690910D06049731
:1068F00011F580911706909118068130910561F08D
:1069000018F0029789F017C04EE150E060EE70E099
:10691000CE010E94CB490FC04EE150E064EC70E024
:10692000CE010E94CB4907C04EE150E068EA70E01A
:10693000CE010E94CB4980910C0690910D060597DF
:1069400011F580911706909118068130910561F03C
:1069500018F0029789F017C04EE150E06CE870E043
:10696000CE010E94CB490FC04EE150E060E770E0DD
:10697000CE010E94CB4907C04EE150E064E570E0D3
:10698000CE010E94CB4980910C0690910D0606978E
:1069900011F580911706909118068130910561F0EC
:1069A00018F0029789F017C04EE150E068E370E0FC
:1069B000CE010E94CB490FC04EE150E06CE170E087
:1069C000CE010E94CB4907C04EE150E060E070E08C
:1069D000CE010E94CB498FE190E00E941D0680917C
:1069E0000C0690910D06892B09F47AD180910C0642
:1069F00090910D06019711F40E94E53F80910C06DD
:106A000090910D06029711F40E94074180910C06A7
:106A100090910D06049711F40E94234280910C0678
:106A200090910D06059711F40E94902880910C0614
:106A300090910D06069709F432D0809134068111A9
:106A40000CC081E0809377061092410610920106F7
:106A50008FE190E00E941D063AD3D09234062FE7D2
:106A600088E391E0215080409040E1F700C00000B1
:106A700080917706882311F40C94CF2908C0213027
:106A800009F0BCCD77CD213009F024CEDFCDDF91E8
:106A9000CF911F910F91FF90EF90DF900895EF92AB
:106AA000FF920F931F93CF93DF93A8958091410698
:106AB00081110FC18FE190E00E941D060E94680DB8
:106AC0008091650690E0909318068093170685E004
:106AD00080933406809141068111FBC0C1E0D5E06E
:106AE000A8950E94070E809134068230A9F4809107
:106AF0001706909118060196909318068093170632
:106B00000FE110E02CE330E046EE50E069E670E083
:106B100081E090E00E94B404809134068330A9F4AF
:106B2000809117069091180601979093180680930C
:106B300017060FE110E02CE330E046EE50E069E686
:106B400070E081E090E00E94B4048091170690917B
:106B500018068330910528F0109218061092170637
:106B600007C08130910501F118F00297C9F154C0B6
:106B70000F2EFFE7EF2EF4E0FF2EF02D02E02FE1C5
:106B800030E04FEF5FEF6DE770E088E290E00E9449
:106B90009305109265064EE150E068E370E085EEE3
:106BA00095E00E94AE4938C00F2EF5E7EF2EF4E0D5
:106BB000FF2EF02D02E02FE130E04FEF5FEF6DE7A9
:106BC00070E088E290E00E949305C09365064EE174
:106BD00050E06CE170E085EE95E00E94AE491CC08B
:106BE0000F2EFBE6EF2EF4E0FF2EF02D02E02FE15A
:106BF00030E04FEF5FEF6DE770E088E290E00E94D9
:106C0000930582E0809365064EE150E060E070E01D
:106C100085EE95E00E94AE4980913406811110C046
:106C2000A895C093410610921E0610921D06C093AF
:106C30002F068FE190E00E941D06A8950E940E226B
:106C4000809134068130A9F5A895C0934106109231
:106C50001E0610921D06C0932F068FE190E00E9441
:106C60001D06A8951092770680916506813069F01F
:106C700018F0823099F01AC04EE150E068E370E0FD
:106C800085EE95E00E94AE4911C04EE150E06CE106
:106C900070E085EE95E00E94AE4908C04EE150E0FC
:106CA00060E070E085EE95E00E94AE49A8950E94F4
:106CB000AF29D09334062FEF80E792E02150804037
:106CC0009040E1F700C0000080914106882309F45C
:106CD00007CFDF91CF911F910F91FF90EF90089513
:106CE000AF92BF92CF92DF92EF92FF920F931F93DA
:106CF000CF93DF93A895809141068111DDC18FE18B
:106D000090E00E941D060E94680D8091690690E047
:106D1000909318068093170685E08093340680913F
:106D200041068111C9C10F2EF7E0AF2EF02D0F2EB5
:106D3000F6E0BF2EF02DC5E06894CC24C2F80F2EEB
:106D4000F3E0DF2EF02DD1E0A8950E94070E809190
:106D500034068230A9F480911706909118060196A6
:106D600090931806809317060FE110E02CE330E0B3
:106D700046EE50E069E670E081E090E00E94B404E5
:106D8000809134068330A9F48091170690911806FB
:106D9000019790931806809317060FE110E02CE3FB
:106DA00030E046EE50E069E670E081E090E00E945D
:106DB000B404E0911706F0911806E830F10528F0C8
:106DC000109218061092170608C0E830F10508F076
:106DD000E4C0E357FF4F0C94A3460F2EFEE8EF2EBE
:106DE000F4E0FF2EF02D02E02FE130E04FEF5FEFF7
:106DF0006DE770E082E390E00E94930510926906CF
:106E00004EE150E068E672E085EE95E00E94AE4902
:106E1000C4C00F2EF9E8EF2EF4E0FF2EF02D02E0B3
:106E20002FE130E04FEF5FEF6DE770E082E390E03D
:106E30000E949305D09369064EE150E06CE472E045
:106E400085EE95E00E94AE49A8C00F2EFFE7EF2E19
:106E5000F4E0FF2EF02D02E02FE130E04FEF5FEF86
:106E60006DE770E088E290E00E94930582E08093F5
:106E700069064EE150E060E372E085EE95E00E9425
:106E8000AE498BC00F2EF5E7EF2EF4E0FF2EF02D6C
:106E900002E02FE130E04FEF5FEF6DE770E088E256
:106EA00090E00E949305D09269064EE150E064E1C3
:106EB00072E085EE95E00E94AE496FC00F2EFBE6B2
:106EC000EF2EF4E0FF2EF02D02E02FE130E04FEF47
:106ED0005FEF6DE770E088E290E00E949305C0925A
:106EE000690644E150E068EF71E085EE95E00E94AC
:106EF000AE4953C00F2EF1E6EF2EF4E0FF2EF02D39
:106F000002E02FE130E04FEF5FEF6DE770E088E2E5
:106F100090E00E949305C09369064EE150E06CED4D
:106F200071E085EE95E00E94AE4937C00F2EF7E57F
:106F3000EF2EF4E0FF2EF02D02E02FE130E04FEFD6
:106F40005FEF6DE770E088E290E00E949305B092F9
:106F500069064EE150E060EC71E085EE95E00E943C
:106F6000AE491BC00F2EFDE4EF2EF4E0FF2EF02DF6
:106F700002E02FE130E04FEF5FEF6DE770E088E275
:106F800090E00E949305A09269064EE150E064EA09
:106F900071E085EE95E00E94AE4980913406811142
:106FA0000FC0A895D093410610921E0610921D06A0
:106FB000D0932F068FE190E00E941D060E940E22C2
:106FC00080913406813009F066C0A895D0934106BF
:106FD00010921E0610921D06D0932F068FE190E0AE
:106FE0000E941D0610927706E09169068E2F90E0B0
:106FF0008830910508F04CC0FC01EB56FF4F0C9413
:10700000A3464EE150E068E672E085EE95E00E940E
:10701000AE493EC04EE150E06CE472E085EE95E092
:107020000E94AE4935C04EE150E060E372E085EE6B
:1070300095E00E94AE492CC04EE150E064E172E060
:1070400085EE95E00E94AE4923C04EE150E068EF26
:1070500071E085EE95E00E94AE491AC04EE150E025
:107060006CED71E085EE95E00E94AE4911C04EE1F5
:1070700050E060EC71E085EE95E00E94AE4908C0FA
:107080004EE150E064EA71E085EE95E00E94AE4981
:10709000A8950E94AF29C0933406A8952FEF80E7EA
:1070A00092E0215080409040E1F700C000008091C4
:1070B0004106882309F448CEDF91CF911F910F91AB
:1070C000FF90EF90DF90CF90BF90AF9008959F9288
:1070D000AF92BF92CF92DF92EF92FF920F931F93E6
:1070E000CF93DF9380910106811163C78FE190E018
:1070F0000E941D060E946F0E1092640685E0809328
:10710000340680910106811154C7C5EED5E00F2EDB
:10711000F8E5AF2EF2E0BF2EF02D0F2EFAE5CF2EC0
:10712000D12CF02D0F2EF5E09F2EF02DE09163066F
:107130008E2F90E08E30910508F026C7FC01E356B3
:10714000FF4F0C94A3460F2EF5E2EF2EF4E0FF2E36
:10715000F02D01E02FE130E04FEF5FEF62E370E0F0
:107160008FE090E00E9493050F2EFEE1EF2EF4E0F9
:10717000FF2EF02D2FE130E04FEF5FEF66E470E07F
:107180008CE390E00E949305E880F98003E02FE112
:1071900030E040E058EF62E870E080E590E00E9467
:1071A000E305888199819093D9058093D8050E9441
:1071B000070E809134068230A9F48091D805909111
:1071C000D90501969093D9058093D8050FE110E079
:1071D0002CE330E046EE50E069E670E081E090E0BC
:1071E0000E94B404809134068330A9F48091D805BC
:1071F0009091D90501979093D9058093D8050FE117
:1072000010E02CE330E046EE50E069E670E081E00B
:1072100090E00E94B4048091D8059091D9058F35F3
:10722000914020F01092D9051092D8058091D80590
:107230009091D905998388838FE798E321E0815065
:1072400090402040E1F700C000009EC60F2EF6E0FF
:10725000EF2EF4E0FF2EF02D01E02FE130E04FEFB4
:107260005FEF62E370E08FE090E00E9493050F2EE5
:10727000F8EFEF2EF3E0FF2EF02D2FE130E04FEF8F
:107280005FEF66E470E08CE390E00E949305EA8093
:10729000FB8003E02FE130E040E058EF62E870E06F
:1072A00080E590E00E94E3058A819B8190932C0603
:1072B00080932B060E94070E809134068230A9F439
:1072C00080912B0690912C06019690932C0680932A
:1072D0002B060FE110E02CE330E046EE50E069E6CB
:1072E00070E081E090E00E94B40480913406833025
:1072F000A9F480912B0690912C06019790932C066F
:1073000080932B060FE110E02CE330E046EE50E0D6
:1073100069E670E081E090E00E94B40480912B0661
:1073200090912C06853F914020F010922C061092EF
:107330002B0680912B0690912C069B838A838FE7E6
:1073400098E321E0815090402040E1F700C0000028
:107350001BC60F2EF0EEEF2EF3E0FF2EF02D01E016
:107360002FE130E04FEF5FEF62E370E08FE090E0FD
:107370000E9493050F2EF8ECEF2EF3E0FF2EF02D78
:107380002FE130E04FEF5FEF66E470E08FE090E0D8
:107390000E949305EC80FD8003E02FE130E040E0A7
:1073A00058EF62E870E080E590E00E94E3058C8190
:1073B0009D8190937206809371060E94070E8091C2
:1073C00034068230A9F4809171069091720601967C
:1073D00090937206809371060FE110E02CE330E089
:1073E00046EE50E069E670E081E090E00E94B4046F
:1073F000809134068330A9F48091710690917206D1
:10740000019790937206809371060FE110E02CE3D0
:1074100030E046EE50E069E670E081E090E00E94E6
:10742000B40480917106909172068F31910538F005
:107430008FE090E0909372068093710608C00F97DA
:1074400030F48FE090E09093720680937106809103
:107450007106909172069D838C838FE798E321E0FB
:10746000815090402040E1F700C000008DC50F2EF4
:10747000F0EBEF2EF3E0FF2EF02D01E02FE130E0F6
:107480004FEF5FEF62E370E08FE090E00E949305C2
:107490000F2EF8E9EF2EF3E0FF2EF02D2FE130E074
:1074A0004FEF5FEF66E470E08FE090E00E9493059D
:1074B000EE80FF8003E02FE130E040E058EF62E82B
:1074C00070E080E590E00E94E3058E819F819093BB
:1074D0001406809313060E94070E809134068230B2
:1074E000A9F48091130690911406019690931406C6
:1074F000809313060FE110E02CE330E046EE50E0FD
:1075000069E670E081E090E00E94B4048091340666
:107510008330A9F4809113069091140601979093FB
:107520001406809313060FE110E02CE330E046EEE2
:1075300050E069E670E081E090E00E94B404809140
:107540001306909114068F31910538F08FE090E08A
:10755000909314068093130608C00F9730F48FE0C1
:1075600090E09093140680931306809113069091F7
:1075700014069F838E838FE798E321E0815090402B
:107580002040E1F700C00000FFC40F2EF0E8EF2E0E
:10759000F3E0FF2EF02D01E02FE130E04FEF5FEF41
:1075A0006CE370E08FE090E00E94930588859985F8
:1075B000019789F40F2EFDE3EF2EF5E0FF2EF02D5D
:1075C00003E02FE130E040E058EF62E870E080E552
:1075D00090E00E94930588859985892B89F40F2E68
:1075E000F8E3EF2EF5E0FF2EF02D03E02FE130E081
:1075F00040E058EF62E870E080E590E00E9493057B
:107600008885809340060E94070E80913406823060
:1076100089F4809140068F5F809340060FE110E06F
:107620002CE330E046EE50E069E670E081E090E067
:107630000E94B40480913406833089F4809140061E
:107640008150809340060FE110E02CE330E046EEDD
:1076500050E069E670E081E090E00E94B40480911F
:107660004006823010F0109240068091400690E073
:10767000998788878FE798E321E0815090402040E8
:10768000E1F700C0000080C40F2EF8E6EF2EF3E013
:10769000FF2EF02D01E02FE130E04FEF5FEF62E3CE
:1076A00070E08FE090E00E9493050F2EF0E5EF2E42
:1076B000F3E0FF2EF02D2FE130E04FEF5FEF66E4B7
:1076C00070E08FE090E00E949305EA84FB8403E081
:1076D00020E038EF4FEF5FEF62E870E080E590E088
:1076E0000E94E3058A859B8590931206809311067C
:1076F0000E94070E809134068230A9F48091110611
:1077000090911206019690931206809311060FE154
:1077100010E02CE330E046EE50E069E670E081E0F6
:1077200090E00E94B404809134068330A9F48091E3
:1077300011069091120601979093120680931106FC
:107740000FE110E02CE330E046EE50E069E670E037
:1077500081E090E00E94B40480911106909112069D
:107760008B3F910520F01092120610921106809125
:107770001106909112069B878A878FE798E321E094
:10778000815090402040E1F700C00000FDC30F2E63
:10779000F8E3EF2EF3E0FF2EF02D01E02FE130E0D3
:1077A0004FEF5FEF62E370E08FE090E00E9493059F
:1077B0000F2EF0E2EF2EF3E0FF2EF02D2FE130E060
:1077C0004FEF5FEF66E470E08FE090E00E9493057A
:1077D000EC84FD8403E02FE130E040E058EF62E804
:1077E00070E080E590E00E94E3058C859D85909394
:1077F0002406809323060E94070E8091340682306F
:10780000A9F4809123069091240601969093240672
:10781000809323060FE110E02CE330E046EE50E0C9
:1078200069E670E081E090E00E94B4048091340643
:107830008330A9F4809123069091240601979093B8
:107840002406809323060FE110E02CE330E046EE9F
:1078500050E069E670E081E090E00E94B40480911D
:107860002306909124068536910520F01092240677
:107870001092230680912306909124069D878C8781
:107880008FE798E321E0815090402040E1F700C06D
:1078900000007AC30F2EF8E0EF2EF3E0FF2EF02D5C
:1078A00001E02FE130E04FEF5FEF62E370E08FE047
:1078B00090E00E9493050F2EF0EFEF2EF2E0FF2EE6
:1078C000F02D2FE130E04FEF5FEF66E470E08FE0E6
:1078D00090E00E949305EE84FF8403E02FE130E006
:1078E00040E058EF62E870E080E590E00E94E30538
:1078F0008E859F8590932206809321060E94070E15
:10790000809134068230A9F480912106909122065C
:10791000019690932206809321060FE110E02CE35C
:1079200030E046EE50E069E670E081E090E00E94D1
:10793000B404809134068330A9F48091210690919B
:107940002206019790932206809321060FE110E012
:107950002CE330E046EE50E069E670E081E090E034
:107960000E94B404809121069091220685369105EB
:1079700020F010922206109221068091210690910B
:1079800022069F878E878FE798E321E08150904001
:107990002040E1F700C00000F7C20F2EF0E7EF2E05
:1079A000F2E0FF2EF02D01E02FE130E04FEF5FEF2E
:1079B0006CE370E08FE090E00E949305E88CF98C16
:1079C00003E02FE130E040E058EF62E870E080E54E
:1079D00090E00E94E305888D998D909360068093D6
:1079E0005F060E94070E809134068230A9F48091D0
:1079F0005F069091600601969093600680935F0603
:107A00000FE110E02CE330E046EE50E069E670E074
:107A100081E090E00E94B404809134068330A9F4A0
:107A200080915F0690916006019790936006809325
:107A30005F060FE110E02CE330E046EE50E069E62F
:107A400070E081E090E00E94B40480915F06909124
:107A50006006893C910528F0D0926006C0925F06CE
:107A600007C08A35910520F4D0926006C0925F0667
:107A700080915F0690916006998F888F8FE798E3D9
:107A800021E0815090402040E1F700C000007CC21E
:107A90000F2EF6ECEF2EF2E0FF2EF02D01E02FE19D
:107AA00030E04FEF5FEF6CE370E08FE090E00E941A
:107AB0009305EA8CFB8C03E02FE130E040E058EFC7
:107AC00062E870E080E590E00E94E3058A8D9B8D7E
:107AD0009093E4058093E3050E94070E809134069D
:107AE0008230A9F48091E3059091E405019690938A
:107AF000E4058093E3050FE110E02CE330E046EE6F
:107B000050E069E670E081E090E00E94B40480916A
:107B100034068330A9F48091E3059091E405019740
:107B20009093E4058093E3050FE110E02CE330E04F
:107B300046EE50E069E670E081E090E00E94B40417
:107B40008091E3059091E405C39720F01092E4053D
:107B50001092E3058091E3059091E4059B8F8A8F55
:107B60008FE798E321E0815090402040E1F700C08A
:107B700000000AC20F2EFEEDEF2EF2E0FF2EF02DD8
:107B800001E02FE130E04FEF5FEF6CE370E08EE15A
:107B900090E00E94930588899989019789F40F2EB6
:107BA000FDE3EF2EF5E0FF2EF02D03E02FE130E0B6
:107BB00040E058EF62E870E080E590E00E949305B5
:107BC00088899989892B89F40F2EF8E3EF2EF5E047
:107BD000FF2EF02D03E02FE130E040E058EF62E8A7
:107BE00070E080E590E00E94930588898093D40539
:107BF0000E94070E80913406823089F48091D4056A
:107C00008F5F8093D4050FE110E02CE330E046EE67
:107C100050E069E670E081E090E00E94B404809159
:107C20003406833089F48091D40581508093D40543
:107C30000FE110E02CE330E046EE50E069E670E042
:107C400081E090E00E94B4048091D405823010F06D
:107C50001092D4058091D40590E0998B888B8FE7A2
:107C600098E321E0815090402040E1F700C00000FF
:107C70008BC18091D405811103C01092630684C129
:107C8000813009F081C10F2EF8E6EF2EF3E0FF2ED0
:107C9000F02D01E02FE130E04FEF5FEF62E370E0A5
:107CA0008FE090E00E9493050F2EF0EBEF2EF2E0B4
:107CB000FF2EF02D2FE130E04FEF5FEF66E470E034
:107CC0008FE090E00E949305EA88FB8803E02FE1B3
:107CD00030E040E058EF62E870E080E590E00E941C
:107CE000E3058A899B8990936206809361060E94CE
:107CF000070E809134068230A9F48091610690913C
:107D00006206019690936206809361060FE110E08F
:107D10002CE330E046EE50E069E670E081E090E070
:107D20000E94B404809134068330A9F480916106E6
:107D300090916206019790936206809361060FE12D
:107D400010E02CE330E046EE50E069E670E081E0C0
:107D500090E00E94B40480916106909162068B3F8E
:107D6000910520F0109262061092610680916106E2
:107D7000909162069B8B8A8B8FE798E321E081507C
:107D800090402040E1F700C00000FEC08091D40583
:107D9000811103C010926306F7C0813009F0F4C06E
:107DA0000F2EF9E9EF2EF2E0FF2EF02D01E02FE18A
:107DB00030E04FEF5FEF62E370E08FE090E00E9411
:107DC00093050F2EF6E8EF2EF2E0FF2EF02D2FE1B7
:107DD00030E04FEF5FEF66E470E08FE090E00E94EC
:107DE0009305EC88FD8803E02FE130E040E058EF98
:107DF00062E870E080E590E00E94E3058C899D894F
:107E000090933F0680933E060E94070E80913406B1
:107E10008230A9F480913E0690913F06019690939E
:107E20003F0680933E060FE110E02CE330E046EE83
:107E300050E069E670E081E090E00E94B404809137
:107E400034068330A9F480913E0690913F06019755
:107E500090933F0680933E060FE110E02CE330E064
:107E600046EE50E069E670E081E090E00E94B404E4
:107E700080913E0690913F06C39720F010923F06F6
:107E800010923E0680913E0690913F069D8B8C8B12
:107E90008FE798E321E0815090402040E1F700C057
:107EA000000072C00F2EF9E4EF2EF2E0FF2EF02D4D
:107EB00001E02FE130E04FEF5FEF6CE370E08FE027
:107EC00090E00E949305EC8CFD8C03E02FE130E004
:107ED00040E058EF62E870E080E590E00E94E30542
:107EE0008C8D9D8D90930706809306060E94070E49
:107EF000809134068230A9F480910606909107069D
:107F0000019690930706809306060FE110E02CE39C
:107F100030E046EE50E069E670E081E090E00E94DB
:107F2000B404809134068330A9F4809106069091C0
:107F30000706019790930706809306060FE110E06D
:107F40002CE330E046EE50E069E670E081E090E03E
:107F50000E94B4048091E3059091E4058935924034
:107F600020F0B0920706A092060680910606909136
:107F700007069D8F8C8F8FE798E321E0815090401A
:107F80002040E1F700C0000080913406813051F4B8
:107F900080930106109277068FE190E00E941D0603
:107FA0000E94AF299092340680910106882309F43B
:107FB000BDC8DF91CF911F910F91FF90EF90DF909F
:107FC000CF90BF90AF909F900895EF92FF920F9344
:107FD0001F93CF93DF93A89580914106811110C123
:107FE0008FE190E00E941D060E94680D80911506A9
:107FF00090E0909318068093170685E080933406EE
:10800000809141068111FCC0C1E0D5E0A8950E9495
:10801000070E809134068230A9F480911706909162
:108020001806019690931806809317060FE110E04A
:108030002CE330E046EE50E069E670E081E090E04D
:108040000E94B404809134068330A9F4809117060D
:1080500090911806019790931806809317060FE1E8
:1080600010E02CE330E046EE50E069E670E081E09D
:1080700090E00E94B404809117069091180603972F
:1080800020F01092180610921706A89580911706F6
:10809000909118068130910501F118F00297C9F10D
:1080A00054C00F2EFFE7EF2EF4E0FF2EF02D02E07C
:1080B0002FE130E04FEF5FEF6DE770E088E290E096
:1080C0000E949305109215064EE150E068E871E0B9
:1080D00085EE95E00E94AE4938C00F2EF5E7EF2EF1
:1080E000F4E0FF2EF02D02E02FE130E04FEF5FEFE4
:1080F0006DE770E088E290E00E949305C09315065A
:108100004EE150E06CE671E085EE95E00E94AE49EC
:108110001CC00F2EFBE6EF2EF4E0FF2EF02D02E048
:108120002FE130E04FEF5FEF6DE770E088E290E025
:108130000E94930582E0809315064EE150E060E5D1
:1081400071E085EE95E00E94AE4980913406811180
:108150000FC0A895C093410610921E0610921D06EE
:10816000C0932F068FE190E00E941D060E940E2210
:10817000809134068130A1F5A895C09341061092F4
:108180001E0610921D06C0932F068FE190E00E94FC
:108190001D061092770680911506813069F018F05F
:1081A000823099F01AC04EE150E068E871E085EE47
:1081B00095E00E94AE4911C04EE150E06CE671E0DE
:1081C00085EE95E00E94AE4908C04EE150E060E5C2
:1081D00071E085EE95E00E94AE49A8950E94AF2916
:1081E000D09334062FEF80E792E0215080409040FA
:1081F000E1F700C0000080914106882309F406CF12
:10820000DF91CF911F910F91FF90EF900895EF9222
:10821000FF920F931F93CF93DF93A8958091410610
:1082200081110AC18FE190E00E941D060E94680D35
:1082300080911C0690E0909318068093170685E0C5
:1082400080933406809141068111F6C0C1E0D5E0EB
:10825000A8950E94070E809134068230A9F480917F
:1082600017069091180601969093180680931706AA
:108270000FE110E02CE330E046EE50E069E670E0FC
:1082800081E090E00E94B404809134068330A9F428
:108290008091170690911806019790931806809385
:1082A00017060FE110E02CE330E046EE50E069E6FF
:1082B00070E081E090E00E94B404809117069091F4
:1082C00018068330910528F01092180610921706B0
:1082D00007C08130910501F118F00297C9F153C030
:1082E0000F2EFFE7EF2EF4E0FF2EF02D02E02FE13E
:1082F00030E04FEF5FEF6DE770E088E290E00E94C2
:10830000930510921C064EE150E064E371E085EEA7
:1083100095E00E94AE4937C00F2EF5E7EF2EF4E04E
:10832000FF2EF02D02E02FE130E04FEF5FEF6DE721
:1083300070E088E290E00E949305C0931C064EE135
:1083400050E068E171E085EE95E00E94AE491BC007
:108350000F2EFBE6EF2EF4E0FF2EF02D02E02FE1D2
:1083600030E04FEF5FEF6DE770E088E290E00E9451
:10837000930582E080931C064EE150E06CEF70E0C4
:1083800085EE95E0EBD780913406811110C0A89559
:10839000C093410610921E0610921D06C0932F0630
:1083A0008FE190E00E941D06A8950E940E22809108
:1083B0003406813089F5A895C093410610921E06B7
:1083C00010921D06C0932F068FE190E00E941D06BB
:1083D0001092770680911C06813061F018F082308F
:1083E00089F017C04EE150E064E371E085EE95E05E
:1083F000B5D70FC04EE150E068E171E085EE95E041
:10840000ADD707C04EE150E06CEF70E085EE95E02F
:10841000A5D7A8950E94AF29D09334062FEF80E707
:1084200092E0215080409040E1F700C00000809130
:108430004106882309F40CCFDF91CF911F910F9152
:10844000FF90EF900895EF92FF920F931F93CF93B9
:10845000DF93A89580914106811109C18FE190E0D9
:108460000E941D060E94680D8091740690E0909312
:1084700018068093170685E08093340680914106A4
:108480008111F5C0C1E0D5E0A8950E94070E80914A
:1084900034068230A9F4809117069091180601964F
:1084A00090931806809317060FE110E02CE330E05C
:1084B00046EE50E069E670E081E090E00E94B4048E
:1084C000809134068330A9F48091170690911806A4
:1084D000019790931806809317060FE110E02CE3A4
:1084E00030E046EE50E069E670E081E090E00E9406
:1084F000B40480911706909118068330910528F0F6
:10850000109218061092170607C081309105F9F0F5
:1085100018F00297B9F151C00F2EFFE7EF2EF4E0EB
:10852000FF2EF02D02E02FE130E04FEF5FEF6DE71F
:1085300070E088E290E00E949305109274064EE18C
:1085400050E060EE70E085EE95E008D736C00F2E63
:10855000F5E7EF2EF4E0FF2EF02D02E02FE130E002
:108560004FEF5FEF6DE770E088E290E00E949305C7
:10857000C09374064EE150E064EC70E085EE95E047
:10858000EDD61BC00F2EFBE6EF2EF4E0FF2EF02DF4
:1085900002E02FE130E04FEF5FEF6DE770E088E23F
:1085A00090E00E94930582E0809374064EE150E0D3
:1085B00068EA70E085EE95E0D1D6809134068111AD
:1085C00010C0A895C093410610921E0610921D0679
:1085D000C0932F068FE190E00E941D06A8950E948F
:1085E0000E2280913406813091F5A895C093410602
:1085F00010921E0610921D06C0932F068FE190E088
:108600000E941D06A895109277068091740681300D
:1086100061F018F0823089F017C04EE150E060EE52
:1086200070E085EE95E09AD60FC04EE150E064EC24
:1086300070E085EE95E092D607C04EE150E068EA22
:1086400070E085EE95E08AD6A8950E94AF29D09378
:1086500034062FEF80E792E0215080409040E1F710
:1086600000C0000080914106882309F40DCFDF91FE
:10867000CF911F910F91FF90EF9008951F920F924D
:108680000FB60F9211248F939F938CB190E090932B
:108690006C0680936B069F918F910F900FBE0F9089
:1086A0001F9018951F920F920FB60F9211242F93BF
:1086B0008F939F938091DF059091E0050196883E0E
:1086C00023E0920728F49093E0058093DF0504C02F
:1086D0001092E0051092DF0580910806811105C017
:1086E00010926E0610926D060BC0813049F4809195
:1086F0006D0690916E06019690936E0680936D06BE
:1087000080912906811105C01092DE051092DD05C9
:108710000BC0813049F48091DD059091DE05019612
:108720009093DE058093DD0580911F06811105C0C1
:108730001092E2051092E1050BC0813049F480915E
:10874000E1059091E20501969093E2058093E105A1
:108750009F918F912F910F900FBE0F901F901895A2
:108760002FEF89E698E1215080409040E1F700C06A
:1087700000008FEF8ABB81BB8093610081E084BBE6
:1087800088EA8FBD8CE08EBD1DBC1CBC17BC16BC1E
:108790008AE78BBD82E18ABD19BC18BC10927900B2
:1087A00010927800C0E1C7BF10BE87E683BF12BE3B
:1087B00011BE81E880938B0085E080938A0010923F
:1087C000890010928800109281001092800010920F
:1087D00087001092860010928500109284001092FB
:1087E0008300109282001BB888E98AB986E08093E2
:1087F0009500109290008FE289B98FE181BD8FE0E2
:1088000081BD03D181E00E94B7038FE190E00E9417
:108810001D0681E090E090930B0680930A0610926B
:108820001E0610921D0610920D0610920C06109254
:10883000E0051092DF051092260610922506109290
:10884000DC051092090610926F061092020680E570
:1088500090E090936C0680936B06E4E6F0E08081F4
:108860008D7F80837894A49AC5BB2FEF85EA9EE024
:10887000215080409040E1F700C0000015BA84E824
:1088800092E07CD5813079F00E94261EA8950E9446
:10889000C21FA89561E085E892E086D5A89561E0C1
:1088A00084E892E081D5C1E0D0E0A89580910A06E5
:1088B00090910B06019721F4A8950E940E22A8958D
:1088C000A89580910A0690910B06892B71F78091EB
:1088D0006B0690916C068335910599F5D0930B0644
:1088E000C0930A060E9419160FE110E02CE330E055
:1088F00044E650E06BE470E08EE690E00E94B40441
:1089000024E230E04AE550E064E670E088E090E080
:108910000E94B40424E230E04AE550E064E670E0EE
:1089200088E090E00E94B40424E230E04AE550E0A0
:1089300064E670E08FED90E00E94B4040E940E2285
:10894000A8950E9438200E943A16A89503E02FE1CE
:1089500030E04FEF5FEF69E170E085E890E00E9462
:1089600036130E94E41F0E94D51280910A0690914E
:108970000B06019781F5A8950E9419160FE110E0EA
:108980002CE330E044E650E06BE470E08EE690E0EB
:108990000E94B40424E230E04AE550E064E670E06E
:1089A00088E090E00E94B40424E230E04AE550E020
:1089B00064E670E088E090E00E94B40424E230E0D5
:1089C0004AE550E064E670E08FED90E00E94B40468
:1089D0000E940E22A8952FEF81EE94E02150804056
:1089E0009040E1F700C000000E94ED100E940E20B0
:1089F0000E947E110E94F91158CFC098AB9AAF9A8D
:108A00008FB9779BFECF8FB1089587E087BBC09A5F
:108A1000AB9AAF9A83E58DB91EB880E8EEDF80E0AF
:108A2000ECDF80E0EADF8AE18A95F1F700C0089583
:108A3000EF92FF920F931F93CF93DF9300D000D05C
:108A4000CDB7DEB77C018B01A895AB9AAF9A1A829D
:108A500019821C821B8280EDD0DF80E0CEDF8FB1D7
:108A600090E09A83898389819A81982F88279A83B5
:108A7000898380E0C2DF2FB189819A81822B9A831A
:108A8000898389819A8196958795969587959695FC
:108A900087959A83898387EC90E00197F1F700C06E
:108AA000000080E9AADF80E0A8DF8FB190E09C831E
:108AB0008B838B819C81982F88279C838B8380E07C
:108AC0009CDF2FB18B819C81822B9C838B838B813C
:108AD0009C819695879596958795969587959C8385
:108AE0008B8389819A81F701918380838B819C811B
:108AF000F801918380830F900F900F900F90DF917A
:108B0000CF911F910F91FF90EF90089570D088F052
:108B10009F5790F0B92F9927B751A0F0D1F0660F69
:108B2000771F881F991F1AF0BA95C9F712C0B13084
:108B300081F077D0B1E0089574C0672F782F88272F
:108B4000B85F39F0B93FCCF3869577956795B395C3
:108B5000D9F73EF490958095709561957F4F8F4F32
:108B60009F4F0895E89409C097FB3EF49095809537
:108B7000709561957F4F8F4F9F4F9923A9F0F92FE3
:108B800096E9BB279395F695879577956795B79561
:108B9000F111F8CFFAF4BB0F11F460FF1BC06F5F47
:108BA0007F4F8F4F9F4F16C0882311F096E911C059
:108BB000772321F09EE8872F762F05C0662371F07A
:108BC00096E8862F70E060E02AF09A95660F771F8E
:108BD000881FDAF7880F9695879597F9089557FDBE
:108BE0009058440F551F59F05F3F71F04795880F1B
:108BF00097FB991F61F09F3F79F0879508951216B2
:108C000013061406551FF2CF4695F1DF08C016165D
:108C100017061806991FF1CF86957105610508940E
:108C20000895E894BB2766277727CB0197F9089525
:108C30000BD078C069D028F06ED018F0952309F0D9
:108C40005AC05FC01124EECFCADFA0F3959FD1F3C5
:108C5000950F50E0551F629FF001729FBB27F00DEA
:108C6000B11D639FAA27F00DB11DAA1F649F66273F
:108C7000B00DA11D661F829F2227B00DA11D621F8E
:108C8000739FB00DA11D621F839FA00D611D221F48
:108C9000749F3327A00D611D231F849F600D211D2C
:108CA000822F762F6A2F11249F5750408AF0E1F0CF
:108CB00088234AF0EE0FFF1FBB1F661F771F881F18
:108CC00091505040A9F79E3F510570F014C0AACFB3
:108CD0005F3FECF3983EDCF3869577956795B79503
:108CE000F795E7959F5FC1F7FE2B880F911D96952D
:108CF000879597F9089597F99F6780E870E060E09D
:108D000008959FEF80EC089500240A941616170624
:108D100018060906089500240A941216130614066C
:108D200005060895092E0394000C11F4882352F0CF
:108D3000BB0F40F4BF2B11F460FF04C06F5F7F4F87
:108D40008F4F9F4F0895EE0FFF1F0024001C0BBE96
:108D50000790F691E02D0994A29FB001B39FC00146
:108D6000A39F700D811D1124911DB29F700D811D57
:108D70001124911D0895BB274A3031F4992322F420
:108D8000BDE2909581959F4F01C0BB27FB01552700
:108D9000AA27880F991FAA1FA41710F0A41B839558
:108DA0005051B9F7A05DAA3308F0A95DA1930097CF
:108DB00079F7B111B1931192CB0126C2CF93DF9312
:108DC000CDB7DEB7AE014B5F5F4FFA016191719194
:108DD000AF0180917A0690917B0603D0DF91CF910D
:108DE00008952F923F924F925F926F927F928F924F
:108DF0009F92AF92BF92CF92DF92EF92FF920F932A
:108E00001F93CF93DF93CDB7DEB72B970FB6F894B0
:108E1000DEBF0FBECDBF6C017B018A01FC01178252
:108E20001682838181FFBFC1CE0101963C01F6010C
:108E30009381F70193FD859193FF81917F018823B1
:108E400009F4ADC1853239F493FD859193FF819189
:108E50007F01853221F4B60190E0E6D1E8CF912C74
:108E6000212C312CFFE1F315D8F08B3279F038F456
:108E7000803279F08332A1F4232D20611DC08D3220
:108E800061F0803369F4232D216016C0832D826048
:108E9000382EE32DE4603E2E2AC0F32DF8601DC06D
:108EA00037FC2DC020ED280F2A3040F08E32B9F467
:108EB00036FC75C1232D2064322E19C036FE06C043
:108EC0008AE0989E200D1124922E11C0EAE02E9E79
:108ED000200D1124222EF32DF0623F2E08C08C3677
:108EE00021F4832D8068382E02C0883641F4F701C2
:108EF00093FD859193FF81917F018111B3CF982FCD
:108F00009F7D9554933028F40C5F1F4F9FE3998306
:108F10000DC0833631F0833771F0833509F055C0C9
:108F200020C0F801808189830E5F1F4F88248394BD
:108F3000912C530112C02801F2E04F0E511CF80190
:108F4000A080B18036FE03C0692D70E002C06FEFD3
:108F50007FEFC5014ED14C018201F32DFF773F2EEB
:108F600015C0280122E0420E511CF801A080B180FA
:108F700036FE03C0692D70E002C06FEF7FEFC501C0
:108F80002DD14C01F32DF0683F2E820133FC19C026
:108F9000822D90E088169906A0F4B60180E290E058
:108FA00043D12A94F5CFF50137FC859137FE8191A5
:108FB0005F01B60190E038D121102A9421E0821A95
:108FC00091088114910479F7E1C0843611F0893653
:108FD00039F5F80137FE07C0608171818281938184
:108FE0000C5F1F4F08C060817181072E000C880B39
:108FF000990B0E5F1F4FF32DFF763F2E97FF09C091
:1090000090958095709561957F4F8F4F9F4FF06839
:109010003F2E2AE030E0A30143D1882E861844C0B9
:10902000853731F4232D2F7EB22E2AE030E025C083
:10903000932D997FB92E8F36C1F018F4883579F0C9
:10904000AEC0803719F0883721F0A9C0E92FE06160
:10905000BE2EB4FE0DC0FB2DF460BF2E09C034FE41
:109060000AC0292F2660B22E06C028E030E005C0D5
:1090700020E130E002C020E132E0F801B7FE07C095
:1090800060817181828193810C5F1F4F06C0608176
:10909000718180E090E00E5F1F4FA30101D1882E07
:1090A0008618FB2DFF773F2E36FE0DC0232D2E7F19
:1090B000A22E891458F434FE0BC032FC09C0832D53
:1090C0008E7EA82E05C0B82CA32C03C0B82C01C0DE
:1090D000B92CA4FE0FC0FE01E80DF11D8081803384
:1090E00021F49A2D997EA92E09C0A2FE06C0B39440
:1090F000B39404C08A2D867809F0B394A3FC10C001
:10910000A0FE06C0B21480F4280C922C9B180DC04F
:10911000B21458F4B60180E290E086D0B394F8CF50
:10912000B21418F42B1802C0982C212CA4FE0FC0E6
:10913000B60180E390E078D0A2FE16C0A1FC03C087
:1091400088E790E002C088E590E0B6010CC08A2D67
:10915000867851F0A1FE02C08BE201C080E2A7FC3C
:109160008DE2B60190E060D0891430F4B60180E35E
:1091700090E05AD09A94F8CF8A94F301E80DF11D4B
:109180008081B60190E050D08110F6CF222009F402
:109190004ECEB60180E290E047D02A94F7CFF60198
:1091A0008681978102C08FEF9FEF2B960FB6F894C0
:1091B000DEBF0FBECDBFDF91CF911F910F91FF900A
:1091C000EF90DF90CF90BF90AF909F908F907F9067
:1091D0006F905F904F903F902F900895FC01059005
:1091E000615070400110D8F7809590958E0F9F1FA9
:1091F0000895FC016150704001900110D8F78095EE
:1092000090958E0F9F1F0895DC01FC01672F7191CF
:109210007723E1F7329704C07C916D93708362915C
:10922000AE17BF07C8F308950F931F93CF93DF9333
:10923000FB01238121FD03C08FEF9FEF2CC022FF94
:1092400016C046815781248135814217530744F463
:10925000A081B1819D012F5F3F4F318320838C938B
:10926000268137812F5F3F4F3783268314C08B01C0
:10927000EC01FB010084F185E02D0995892BE1F6D5
:10928000D80116968D919C911797019617969C93ED
:109290008E931697CE01DF91CF911F910F91089574
:1092A000FA01AA27283051F1203181F1E8946F9317
:1092B0006E7F6E5F7F4F8F4F9F4FAF4FB1E03ED0BD
:1092C000B4E03CD0670F781F891F9A1FA11D680F5B
:1092D000791F8A1F911DA11D6A0F711D811D911D8E
:1092E000A11D20D009F468943F912AE0269F112403
:1092F0003019305D3193DEF6CF010895462F477067
:10930000405D4193B3E00FD0C9F7F6CF462F4F70C1
:10931000405D4A3318F0495D31FD4052419302D01F
:10932000A9F7EACFB4E0A6959795879577956795C5
:10933000BA95C9F700976105710508959B01AC01C5
:109340000A2E06945795479537952795BA95C9F7EC
:10935000620F731F841F951FA01D0895DC01CB01B0
:10936000FC01E199FECF06C0FFBBEEBBE09A31964F
:109370000DB20D9241505040B8F70895E199FECFDB
:109380009FBB8EBBE09A99278DB30895A8E1B0E00A
:1093900042E050E0E5CFDC01CB0102C02D9105D0C9
:1093A00041505040D8F70895262FE199FECF9FBB3A
:1093B0008EBB2DBB0FB6F894E29AE19A0FBE0196D0
:0C93C0000895F2DF272FF1CFF894FFCFC3
:1093CC000000000200000000E807000000005754F5
:1093DC003D2025750A47530047533D2025750A53F8
:1093EC004E00534E3D2025750A454E4400574B3DCB
:1093FC002025750A565000503D332E360A52005225
:10940C004C3D2025750A68004F3D73740A53004784
:10941C003D73740A530053523D53746174696F6EFB
:10942C00200A57500057503D536E36332F5062333D
:10943C00370A57540057503D536E41670A57540032
:10944C0057503D50726F66696C65300A575400571F
:10945C00503D50726F66696C65310A575400575015
:10946C003D50726F66696C65320A57540057503D17
:10947C0050726F66696C65330A57540057503D50F3
:10948C00726F66696C65340A57540057503D5072C0
:10949C006F66696C65350A57540053523D555068D8
:1094AC006561746572200A57500053523D507265C5
:1094BC00686561746572200A57500053523D4D61C6
:1094CC006E75616C200A57500053523D5265626FA5
:1094DC006C6C696E67200A57500053523D436869A3
:1094EC007068656174696E67200A57500053523D6D
:1094FC0050434268656174696E67200A5750005387
:10950C00523D5043200A575000202020C2F0E5EC79
:10951C00FF20F0E5E1EEEBEBE8EDE3E0202020208E
:10952C0000C2FBE1E5F0E8F2E520F0E5E6E8EC004E
:10953C00D2E5ECEFE5F0E0F2F3F0E020EFEEEBEE4D
:10954C00F7EAE8202000EDE8E7E020EFF0E820E47F
:10955C00EEEDE0E3F0E5E2E500D2E5ECEFE5F0E07E
:10956C00F2F3F0E020F3E2E5EBE8F7E5EDE8FF00DD
:10957C00202020202020E4EEEDE0E3F0E5E2E020E6
:10958C00202020202000C4EBE8F2E5EBFCEDEEF10E
:10959C00F2FC20E2EFE8F2FBE2E0EDE8FF00D4F3AE
:1095AC00EDEAF6E8FF20E4EEEDEEE3F0E5E2E000B4
:1095BC00EDE8E6EDE5E3EE20EDE0E3F0E5E2E0F2E8
:1095CC00E5EBFF2020202000CCE0EAF1E8ECE0EB1A
:1095DC00FCEDE0FF20ECEEF9EDEEF1F2FC202000CA
:1095EC00E2E5F0F5EDE5E3EE20EDE0E3F0E5E2E0B9
:1095FC00F2E5EBFF20202000CCE0EAF1E8ECE0EB18
:10960C00FCEDE0FF20ECEEF9EDEEF1F2FC20200099
:10961C00E2E5F0F5EDE5E3EE20EDE0E3F0E5E2E088
:10962C00F2E5EBFF20202000D2E5ECEFE5F0E0F2D4
:10963C00F3F0E020E2EAEBFEF7E5EDE8FF20200096
:10964C00CAEEEDF2F0EEEBFC20EFEE20E2E5F0F5E9
:10965C00F320202020202000EDE8E6EDE5E3EE20CD
:10966C00EDE0E3F0E5E2E0F2E5EBFF202020200066
:10967C00CAEEFDF4F4E8F6E8E5EDF220EFF0EEF4D6
:10968C00E8EBFF2020202000E2E5F0F5EDE5E3EE2D
:10969C0020EDE0E3F0E5E2E0F2E5EBFF2020200036
:1096AC00CAEEFDF4F4E8F6E8E5EDF220EFF0EEF4A6
:1096BC00E8EBFF2020202000EDE0E3F0E5E2E0F213
:1096CC00E5EBFF202000D2E5ECEFE5F0E0F2F3F063
:1096DC00E020EDE8E6EDE5E3EE2020202000EFE0D1
:1096EC00E9EAE82000D2E5ECEFE5F0E0F2F3F0E097
:1096FC0020ECE5F1F2E0202020202000C2FBE1E587
:10970C00F0E8F2E520EFF0EEF4E8EBFC00CFF0EE41
:10971C00F4E8EBFC203500CFF0EEF4E8EBFC203461
:10972C0000CFF0EEF4E8EBFC203300CFF0EEF4E8E1
:10973C00EBFC203200CFF0EEF4E8EBFC203100CF54
:10974C00F0EEF4E8EBFC203000536E416700536EF2
:10975C00506200CAEEECEFFCFEF2E5F000C4EEEF56
:10976C002E20EDE0F1F2F0EEE9EAE800EFEBE0F2AA
:10977C000020D1F3F8EAE020EFEBE0F22000ECE877
:10978C00EAF0EEF1F5E5EC00D1F3F8EAE000D0E513
:10979C00E1EEEBEBE8EDE32000D0F3F7EDEEE900C2
:1097AC002020D0F3F7EDEEE920202000CDE8E6ED07
:1097BC00E8E920EDE0E3F02E2000C2E5F0F5EDE85D
:1097CC00E920EDE0E3F02E002020D1F2E0EDF6E808
:1097DC00FF00E2E5F0F5E000EDE8E7E000CCEEF9A3
:1097EC00EDEEF1F2FC00CFF0E8EDFFF2EE20200000
:1097FC00C2DBC1D0C0D2DC00C2DBCACB00C2CACB38
:10980C0000CDE0F1F2F0EEE8F2FC00C7E2F3EAEE94
:10981C00E2FBE520F1E8E3EDE0EBFB00CFF0E5E463
:10982C00F3F1F2E0EDEEE2EAE800D3ECEEEBF7E078
:10983C00EDE8FF00C2F0E5ECFF20EFE0E9EAE8001C
:10984C0020C4E0F2F7E8EA20EDE8E62E20EDE0E3B4
:10985C00F0E5E2E0F2E5EBFF0020C4E0F2F7E8EA25
:10986C0020ECE5F1F2E020EFE0E9EAE800F0F3F7B4
:10987C00EDEEE900EDE8E6EDE8E900EDE0E3F02ED1
:10988C0000C2E5F0F5EDE8E900C2DBD5CEC400007E
:00000001FF
